:020000040800F2
:1000000000060020F50500086525000819250008F0
:10001000412500081925000839250008F7050008C2
:10002000F7050008F7050008F705000895600008C7
:10003000F7050008F7050008F7050008F7050008B0
:10004000F7050008F7050008F7050008F7050008A0
:10005000F7050008F705000881640008AD64000892
:10006000D96400080565000831650008F705000837
:10007000F7050008F7050008F7050008F705000870
:10008000F7050008F7050008F7050008F705000860
:10009000F7050008F7050008F70500085D6500088A
:1000A000F7050008F7050008F7050008F705000840
:1000B000F7050008F7050008F7050008F705000830
:1000C000F7050008F7050008F7050008F705000820
:1000D000F7050008F7050008F7050008F705000810
:1000E000C1650008F7050008F7050008F7050008D6
:1000F000F7050008F7050008F7050008F7050008F0
:10010000F7050008F70500085D660008F705000818
:10011000F7050008F7050008F7050008F7050008CF
:10012000F7050008F7050008F7050008F7050008BF
:10013000F7050008F7050008F7050008F7050008AF
:10014000F7050008F7050008F7050008F70500089F
:10015000F7050008F7050008F7050008F70500088F
:10016000F7050008F7050008F7050008F70500087F
:10017000F705000831580008F7050008F7050008E2
:10018000F7050008F705000849660008F7050008AC
:10019000F7050008F7050008F7050008F70500084F
:1001A000F7050008F7050008F7050008F70500083F
:1001B00035660008F7050008F7050008F705000890
:1001C000F7050008F7050008F7050008F70500081F
:1001D000F70500081D580008F7050008F705000896
:1001E000F7050008F7050008F7050008F7050008FF
:1001F000F7050008F7050008F7050008F7050008EF
:10020000F7050008F7050008F7050008F7050008DE
:10021000F7050008F7050008F7050008F7050008CE
:10022000F7050008F70500087D4C0008F7050008F1
:10023000F7050008F7050008F7050008F7050008AE
:10024000F7050008F7050008F7050008F70500089E
:10025000F7050008F7050008F7050008F70500088E
:10026000F7050008F7050008F7050008F70500087E
:10027000F7050008F7050008F7050008F70500086E
:10028000F7050008F7050008F7050008F70500085E
:10029000F7050008F7050008F7050008F70500084E
:1002A000F7050008F7050008F7050008F70500083E
:1002B000F7050008F7050008F7050008F70500082E
:1002C000F7050008F7050008F7050008F70500081E
:1002D000F7050008F7050008F7050008F70500080E
:1002E000D9070008DD210008ED2400080000000007
:1002F00053B94AB9002908BF00281CBF4FF0FF318D
:100300004FF0FF3000F074B9ADF1080C6DE904CE88
:1003100000F006F8DDF804E0DDE9022304B07047E0
:100320002DE9F047089D04468E46002B4DD18A42A8
:10033000944669D9B2FA82F252B101FA02F3C2F1DB
:10034000200120FA01F10CFA02FC41EA030E94406C
:100350004FEA1C48210CBEFBF8F61FFA8CF708FB8D
:1003600016E341EA034306FB07F199420AD91CEB65
:10037000030306F1FF3080F01F81994240F21C8197
:10038000023E63445B1AA4B2B3FBF8F008FB1033DF
:1003900044EA034400FB07F7A7420AD91CEB040414
:1003A00000F1FF3380F00A81A74240F207816444E4
:1003B000023840EA0640E41B00261DB1D440002369
:1003C000C5E900433146BDE8F0878B4209D9002DCD
:1003D00000F0EF800026C5E9000130463146BDE857
:1003E000F087B3FA83F6002E4AD18B4202D38242C1
:1003F00000F2F980841A61EB030301209E46002D70
:10040000E0D0C5E9004EDDE702B9FFDEB2FA82F2C4
:10041000002A40F09280A1EB0C014FEA1C471FFA22
:100420008CFE0126200CB1FBF7F307FB131140EA09
:1004300001410EFB03F0884208D91CEB010103F1D6
:10044000FF3802D2884200F2CB804346091AA4B298
:10045000B1FBF7F007FB101144EA01440EFB00FE6C
:10046000A64508D91CEB040400F1FF3102D2A645D1
:1004700000F2BB800846A4EB0E0440EA03409CE770
:10048000C6F12007B34022FA07FC4CEA030C20FA1D
:1004900007F401FA06F31C43F9404FEA1C4900FA3D
:1004A00006F3B1FBF9F8200C1FFA8CFE09FB1811BA
:1004B00040EA014108FB0EF0884202FA06F20BD92D
:1004C0001CEB010108F1FF3A80F08880884240F27D
:1004D0008580A8F102086144091AA4B2B1FBF9F0C1
:1004E00009FB101144EA014100FB0EFE8E4508D9BC
:1004F0001CEB010100F1FF346CD28E456AD9023841
:10050000614440EA0840A0FB0294A1EB0E01A14225
:10051000C846A64656D353D05DB1B3EB080261EB93
:100520000E0101FA07F722FA06F3F1401F43C5E96D
:10053000007100263146BDE8F087C2F12003D840A3
:100540000CFA02FC21FA03F3914001434FEA1C47E5
:100550001FFA8CFEB3FBF7F007FB10360B0C43EAD7
:10056000064300FB0EF69E4204FA02F408D91CEB87
:10057000030300F1FF382FD29E422DD90238634485
:100580009B1B89B2B3FBF7F607FB163341EA034125
:1005900006FB0EF38B4208D91CEB010106F1FF3874
:1005A00016D28B4214D9023E6144C91A46EA00466B
:1005B00038E72E46284605E70646E3E61846F8E6FD
:1005C0004B45A9D2B9EB020864EB0C0E0138A3E746
:1005D0004646EAE7204694E74046D1E7D0467BE727
:1005E000023B614432E7304609E76444023842E79F
:1005F000704700BF02E000F000F8FEE772B637482F
:1006000080F30888364880F3098836483649086000
:1006100040F20000CCF200004EF63471CEF2000140
:100620000860BFF34F8FBFF36F8F40F20000C0F23E
:10063000F0004EF68851CEF200010860BFF34F8FF4
:10064000BFF36F8F4FF00000E1EE100A4EF63C71E1
:10065000CEF200010860062080F31488BFF36F8F8C
:1006600004F074FA05F074FC4FF055301F491B4A32
:1006700091423CBF41F8040BFAE71D49184A9142E8
:100680003CBF41F8040BFAE71A491B4A1B4B9A423C
:100690003EBF51F8040B42F8040BF8E7002018495C
:1006A000184A91423CBF41F8040BFAE704F08CFA77
:1006B00005F0C4FC144C154DAC4203DA54F8041B8D
:1006C0008847F9E700F050F8114C124DAC4203DABC
:1006D00054F8041B8847F9E704F074BA00060020B8
:1006E000002200200000000808ED00E000000020CB
:1006F00000060020A86E000800220020C82200206A
:10070000C8220020B04A0020E0020008EC020008E5
:10071000EC020008EC0200082DE9F04F2DED108AE4
:10072000C1F80CD0D0F80CD0BDEC108ABDE8F08F29
:10073000002383F311882846A047002003F00CFC17
:10074000FEE703F025FB00DFFEE70000054B10B5D8
:1007500004460360806810B103685B6898472046D0
:1007600010BD00BFB069000870B500F075FD04F061
:1007700013F9054604F0E0F90446B8B9144B9D425C
:1007800016D001339D4241F2883512BF0446002540
:100790000124104E002004F009F9304601F040FB1E
:1007A00040B944F6206003F0DDFBF6E70025F0E7F2
:1007B0000546EEE70CB100F091F800F05DFF00F0A7
:1007C000C7FD284600F046F900F088F8F9E700BFB9
:1007D000010007B0C82200200448054B054A036009
:1007E00000230549836005F093BF00BFC8220020A5
:1007F000B0690008002500204D07000808B500F08A
:1008000073FDA0F120035842584108BD07B50421EB
:1008100001900DEB010000F085FD03B05DF804FBD5
:1008200007B541F21203022101A8ADF8043000F02F
:1008300079FD03B05DF804FB38B5302383F31188EC
:10084000174803680BB103F06BFC0023154A4FF403
:100850007A71134803F05AFC002383F31188124C79
:10086000236813B12368013B2360636813B1636895
:10087000013B63600D4D2B7833B963687BB902206F
:1008800000F030FE322363602B78032B07D16368BE
:100890002BB9022000F026FE4FF47A73636038BD56
:1008A00058230020390800087824002070230020F5
:1008B000084B187003280CD8DFE800F00805020880
:1008C000022000F0FFBD022000F0EABD024B002232
:1008D0005A6070477023002078240020F7B55648EE
:1008E00001A901F01DFC002800F0A380534B544ADD
:1008F0001C461968013100F0998004339342F8D105
:100900006268504B9A4240F291804F4BDB6803F192
:10091000104303F580139A4280F08880002000F095
:1009200031FD0220FFF7C4FF484B0021D3F8E82037
:10093000C3F8E810D3F81021C3F81011D3F8102130
:10094000D3F8EC20C3F8EC10D3F81421C3F8141139
:10095000D3F81421D3F8F020C3F8F010D3F81821FD
:10096000C3F81811D3F81821D3F8802042F00062A0
:10097000C3F88020D3F8802022F00062C3F88020E2
:10098000D3F88020D3F8802042F00072C3F8802092
:10099000D3F8802022F00072C3F88020D3F8803092
:1009A00072B64FF0E023C3F8084DD4E90004BFF35A
:1009B0004F8FBFF36F8F264AC2F88410BFF34F8F5B
:1009C000536923F480335361BFF34F8FD2F88030E3
:1009D00043F6E076C3F3C905C3F34E335B0103EA84
:1009E000060C29464CEA81770139C2F87472F9D2B3
:1009F000203B13F1200FF2D1BFF34F8FBFF36F8F66
:100A0000BFF34F8FBFF36F8F536923F400335361EC
:100A10000023C2F85032BFF34F8FBFF36F8F3023E4
:100A200083F31188854680F308882047024800F048
:100A3000BFFE03B0F0BD00BFC82200200000109030
:100A400020001090FFFF0F90002200200044025869
:100A500000ED00E02DE9F04FB34B9FB02022FF21C5
:100A6000089016A89E68DB68079300F0AFFDAF4AB8
:100A70001378A3B90121AE4811700360302383F3CA
:100A8000118803680BB103F04BFB0023A94A4FF414
:100A90007A71A74803F03AFB002383F31188089B7F
:100AA00013B1A54B089A1A60A44A1378032B03D0FC
:100AB00000231370A04A53600023089DA04F98465E
:100AC0009B46CDE90533012000F0FCFC25B19A4B93
:100AD0001B68002B00F08783002000F005FC0E90BF
:100AE0000E9B002BF2DB012000F0DAFC0E9B213B79
:100AF0001F2BE8D801A252F823F000BF7D0B00089D
:100B0000A50B00083F0C0008C70A0008C70A000828
:100B1000C70A00082B0F000829110008C10F0008A0
:100B2000A7100008CD100008F3100008C70A00083D
:100B300005110008C70A0008711100081D0C000803
:100B4000C70A0008ED110008DD0C0008150E0008AA
:100B5000C70A00081D100008C70A0008C70A0008D5
:100B6000C70A0008C70A0008C70A0008C70A000821
:100B7000C70A0008C70A00083F0C00080220FFF758
:100B80003DFE002840F05B83089B0221069A11A8D5
:100B9000002A08BF1D4641F21233ADF8443000F080
:100BA000C1FB90E74FF47A7000F09EFB041EEBDB74
:100BB0000220FFF723FE0028E6D0013C052C00F2BE
:100BC0004083DFE804F0030A0D10133905230421E4
:100BD00011A8119300F0A6FB17E004215248F9E791
:100BE00004215848F6E704215748F3E74FF01C0961
:100BF000484609F1040900F0C7FB0421119011A82F
:100C000000F090FBB9F12C0FF2D10120059B4FF0C1
:100C1000000B00FA04F41C43E3B2059300F022FD3C
:100C2000B8F1000F05D0059B03F00B030B2B08BF99
:100C30000025FFF7F5FD46E704214448CAE7B8F16F
:100C4000000FA1D0059B03F00B030B2B9CD10220BE
:100C5000FFF7D4FD0446002896D001204FF000088D
:100C600000F090FB0220FFF723FE1FFA88F94846A8
:100C700000F098FB0546B8B10E99484608F1010806
:100C8000A1F140025142514100F09CFB0028ECD1FF
:100C90000546069441F21213022111A8A046ADF8B0
:100CA000443000F03FFB0EE72E46DFF87C80012049
:100CB000FFF7FEFDD8F80830B34207D9304600F000
:100CC00063FB013040F0C0820436F3E700261B4B83
:100CD000A04606941E70184B5E609FE7B8F1000FA7
:100CE0003FF452AF059B03F00B030B2B7FF44CAF8B
:100CF00064210FA800F00CFB814600287FF444AF6C
:100D00000220FFF77BFD044600283FF43DAF3A6A1E
:100D10007B6A0F9953438DF837908B421AD20C4857
:100D200000F0F4FB30E700BF002200207424002014
:100D30005823002039080008782400207023002060
:100D4000C822002004220020082200200C220020BB
:100D5000546800084FF4801AAC48C846BAFBF2FA4F
:100D600000F0D4FBFFF75CFD01210DF1370000F02E
:100D7000D9FA0F9B434541D9002310AA5146384662
:100D8000CDE9103311AB00F017FD002882D001F03F
:100D9000F1FB109B00EB030901210DF1370000F07E
:100DA000C1FA01F0E7FB484520D9384600F03EFF84
:100DB00080B964210F9B96480AF1010A01FB08F1F2
:100DC000B1FBF3F18DF83710C9B200F09FFB3B6A1D
:100DD0009844CEE701F0CEFB119B184448453FF6FE
:100DE00059AF01F0C7FB109B00EB0309109B4FF4B8
:100DF0007A70A3FB000303F0B5F8CDE7642301216B
:100E00000DF13700A0468DF8373000F08BFA002343
:100E1000079303E7B8F1000F3FF4B6AE059B03F06C
:100E20000B030B2B7FF4B0AE0220FFF741FD322005
:100E300000F05AFAB0F1000AFFF6A6AE079BD146C1
:100E400053440993734B099ADB689A423FF69CAE70
:100E5000BAF5807F3FF798AE6F4A0024A2450A9208
:100E60000EDD4FF47A7000F03FFA0E900E9B002BCF
:100E7000FFF68AAE0E9B01340A9A02F8013BEDE7B9
:100E8000C820FFF7BBFC044600283FF47DAE079B5B
:100E90001F2B11D8C3F1200223F0030016AB5E49CB
:100EA0005245184428BF52460A9200F05DFB0A9A48
:100EB000FF21594800F08AFB00239846CDE9103302
:100EC000079B03F580130B93B9F1000F02D1A046E5
:100ED000099B9DE711AB504A0B993846029310AB22
:100EE0004244414401930FAB00934B4601F080F81C
:100EF00000283FF4CFAE01F03FFB0F9B82460A91E2
:100F00009844A9EB030901F037FB109B0A9A13EBF5
:100F10000A0342F10002834272EB0103F3D2384626
:100F200000F084FE0028EED1CEE7B8F1000F3FF4C8
:100F30002BAE059B03F00B030B2B7FF425AE022099
:100F4000FFF7B6FC322000F0CFF9B0F1000AFFF64F
:100F50001BAE1AF003047FF417AE2E4A0AEB060309
:100F6000926893423FF610AEBAF5807F3FF70CAE21
:100F7000DFF8A490A2450DDD4FF47A7000F0B4F9CB
:100F80000E900E9B002BFFF6FFAD0E9B013409F86F
:100F9000013BEFE7C820FFF731FC044600283FF48F
:100FA000F3ADCAF387021C4930464FEAAA0900F0A4
:100FB00015FB804600283FF46DAE06EB89062DE652
:100FC0000220FFF71BFC00283FF4DEAD00F018FA0A
:100FD00000283FF4D9AD4FF00009DFF838A04C46A7
:100FE000DAF808304B450CD9484609F1040900F0FD
:100FF000CBF90422119011A9204601F0F7F804461C
:10100000EEE72046FFF702FC08E600BF796800081B
:10101000916800080022002074230020642110A899
:1010200000F076F9044600287FF4AEAD0220FFF709
:10103000E5FB00283FF4A8AD109BA14603F0030A8E
:101040001099A1EB0A01A1421BD91F2C11D8169BA4
:1010500001330ED024F003031EAA134453F8203C9E
:1010600011934846042211A9043401F0BFF88146C7
:10107000E6E7042311AA04F58011384601F004F8CC
:10108000EFE7BAF1000F0CD0534611AA01F5801119
:10109000384600F0F9FF4846524611A901F0A6F87B
:1010A00081464846AEE70023642111A8119300F061
:1010B0002FF900287FF468AD0220FFF79FFB00287E
:1010C0003FF462AD119800F091F99BE70023642191
:1010D00011A8119300F01CF900287FF455AD0220EF
:1010E000FFF78CFB00283FF44FAD119800F080F91A
:1010F00088E70220FFF782FB00283FF445AD00F0AF
:101100008FF97FE70220FFF779FB00283FF43CAD21
:1011100011A9142000F08AF90990FFF777FB0999CB
:1011200011A800F0FFF879E5322000F0DDF8041E88
:10113000FFF62AADA3077FF427AD444A04EB0B0367
:10114000926893423FF620AD0220FFF757FB00283C
:101150003FF41AAD24F003045C44A3453FF45EADB4
:1011600058460BF1040B00F00FF9FFF74FFBF4E7C3
:101170004FF47A70FFF742FB00283FF405AD00F012
:101180003FF980B1169B013328D011AB16AA4FF45A
:1011900080113846029310AB01930FAB00932023CC
:1011A00000F026FF08B9444674E501F0E5F9284E41
:1011B00004460D4601F0E0F9109B1B1945F10002B1
:1011C000834272EB0103F5D2304600F02FFD002878
:1011D000F0D12022FF2116A800F0F8F9FFF720FB3C
:1011E0001C4802F0BFFE1FB0BDE8F08FB8F1000F41
:1011F0003FF4CAAC059B03F00B030B2B7FF4C4AC8C
:101200000023642111A8119300F082F804460028FD
:101210007FF4BAAC0220FFF7F1FA814600283FF4D0
:10122000B3ACFFF7FDFA41F2883002F09BFE119853
:1012300000F062FAC846254600F014FA43E48046FE
:10124000ECE44FF0000B9FE4069423E5002200201D
:10125000C8220020A0860100704700002DE9F84F49
:101260004FF47A7306460D46002402FB03F7DFF8BD
:101270005080DFF8509098F900305FFA84FA5A1CD9
:1012800001D0A34212D159F824002A4631460368FE
:10129000D3F820B03B46D847854207D1074B012001
:1012A00083F800A0BDE8F88F0124E4E7002CFBD010
:1012B0004FF4FA7002F056FE0020F3E7C424002039
:1012C000102200201422002070B504464FF47A76D4
:1012D000412C254628BF412506FB05F002F042FEC1
:1012E000641BF5D170BD0000002307B50246012143
:1012F0000DF107008DF80730FFF7B0FF20B19DF822
:10130000070003B05DF804FB4FF0FF30F9E7000081
:101310000A46042108B5FFF7A1FF80F00100C0B222
:10132000404208BD074B0A4630B41978064B53F8C3
:101330002140014623682046DD69044BAC4630BCA1
:10134000604700BFC424002014220020A0860100B2
:1013500070B50A4E00240A4D03F022F93080286847
:101360003388834208D903F017F92B68044401330A
:10137000B4F5003F2B60F2D370BD00BFC62400203F
:101380008024002003F092B900F1006000F50030E5
:101390000068704700F10060920000F5003003F033
:1013A0002FB90000054B1A68054B1B889B1A834216
:1013B00002D9104403F0F0B80020704780240020C8
:1013C000C624002038B50446074D29B128682044BA
:1013D000BDE8384003F0ECB82868204403F0E2F898
:1013E0000028F3D038BD00BF8024002000207047C3
:1013F00000F1FF5000F58F10D0F800087047000092
:10140000064991F8243033B100230822086A81F894
:101410002430FFF7BFBF0120704700BF84240020A5
:10142000014B1868704700BF0010005C194B013871
:101430000322084470B51D68174BC5F30B042D0C2F
:101440001E88A6420BD15C680A46013C82421346C4
:101450000FD214F9016F4EB102F8016BF6E7013AB1
:1014600003F10803ECD181420B4602D22C2203F88F
:10147000012B0424094A1688AE4204D1984284BF45
:10148000967803F8016B013C02F10402F3D1581A7B
:1014900070BD00BF0010005C1C220020CC6800085A
:1014A000022804D1054B4FF080629A6170470128F1
:1014B000FCD1034B4FF48032F7E700BF000C025819
:1014C00000180258022804D1044B4FF480629A613C
:1014D0007047012801D1024B98617047000C0258F7
:1014E00000180258022805D1064A536983F4806324
:1014F000536170470128FCD1034A536983F001030B
:10150000F6E700BF000C0258001802580FB4124B47
:1015100030B51A78B5B042B90122104910481A7096
:101520004FF461430B6001F0BBFE39AB0C4C389AB1
:10153000C82102A8019300F0EDFF2368C8280246E5
:10154000DD6902A9074B28BFC8222046A84735B04D
:10155000BDE8304004B07047C8240020CC240020EF
:1015600024250020A0860100002310B5934203D05B
:10157000CC5CC4540133F9E710BD0000013810B54C
:1015800010F9013F3BB191F900409C4203D11AB1DF
:101590000131013AF4E71AB191F90020981A10BD0F
:1015A0001046FCE70138013910F9013F11F9012F0C
:1015B0000BB19342F8D0981A7047000003460246D8
:1015C000D01A12F9011B0029FAD1704702440346D0
:1015D000934202D003F8011BFAE770472DE9F84364
:1015E0001F4D14460746884695F8242052BBDFF865
:1015F00070909CB395F824302BB92022FF214846E7
:101600002F62FFF7E3FF95F824004146C0F108027E
:1016100005EB8000A24228BF2246D6B29200FFF717
:10162000A3FF95F82430A41B17441E449044E4B251
:10163000F6B2082E85F82460DBD1FFF7E1FE002822
:10164000D7D108E02B6A03EB82038342CFD0FFF7A8
:10165000D7FE0028CBD10020BDE8F8830120FBE7AE
:1016600084240020024B1A78024B1A70704700BF86
:10167000C42400201022002038B51A4C1A4D2046F0
:1016800001F0B0FE2946204601F0D8FE2D684FF447
:101690007A70D5F89020D2F8043843F00203C2F8EB
:1016A0000438FFF711FE1149284601F0D5FFD5F89F
:1016B00090200F4DD2F80438286823F002030D491A
:1016C000A042C2F804384FF4E1330B6001D001F0BE
:1016D000E7FD6868A04204D00649BDE8384001F043
:1016E000DFBD38BD002C0020F46B0008FC6B000847
:1016F00014220020AC2400200C4B70B50C4D044685
:101700001E780C4B55F826209A420DD00A4B00212A
:1017100018221846FFF75AFF0460014655F82600C4
:10172000BDE8704001F0BCBD70BD00BFC424002006
:1017300014220020002C0020AC2400208069704777
:10174000C0697047006A7047406A7047806A704796
:10175000F0B5ADF2044D0E46054600214FF47F7200
:1017600001A80091FFF732FF2C6A744301362B6AFF
:101770007343A34216D92B686A46214628465F6800
:101780004FF48063B84770B16A464FF4806312F833
:10179000011BFF290AD1013B9BB2002BF7D104F5B5
:1017A0008064E4E701200DF2044DF0BD0020FAE76B
:1017B00080680368DB69184730B5456A85B0044620
:1017C0008D420FD30568CDE90023026A03ABAD6AF1
:1017D0005143A84720B1206A039BC31A584258417D
:1017E00005B030BD0020FBE7F0B5C56987B0044601
:1017F0008D4212D30C9F866905687143CDE901378C
:1018000005AB00936D69036AA84720B1A069059BE9
:10181000C31A5842584107B0F0BD0020FBE7000052
:10182000F0B5662389B0002405464FF480768068C1
:10183000079403A9CDE90336CDE9054403685B6944
:101840009847A86822462146036800941F692346EA
:10185000B847A8689923079403A9CDE90336CDE9D1
:10186000054403685B699847A868224621460368D7
:1018700000941D692346A84709B0F0BD254B2DE90A
:10188000F04F1B789FB0002504468DF828304FF0AC
:101890009F0E80684FF00123ADF8295005A90995E6
:1018A000CDE905E3CDE9075503685B699847A06872
:1018B00003222946036800922A461E690AABB047F4
:1018C00030B394F88C200C21134B01FB02339DF8AC
:1018D00028101A7991421BD19DF829205B799A42F0
:1018E00016D1A0684FF05A0C0C4B082605A9099692
:1018F000CDE905C3CDE9075503685B699847A06842
:101900002A462946036800961F690AABB84738B9CA
:1019100000204BE13C6800088469000800250001B4
:101920000422B3490AA804F02DFF05460028EFD190
:10193000BDF82C306FF48277A3813B44012BE7D8AC
:10194000079605A9CDE90A00A06803685B69984776
:10195000A0682A462946036800961E690AABB0476C
:101960000028D5D0DDE90A361A0202F4706242EA94
:101970001662FF2ACCD11B0E26F07F465022294644
:10198000142B26610AA828BF1423A373FFF71EFE99
:10199000A068079605A903685B699847A068A37BC0
:1019A000294602689B0000930AAB16692A46B04795
:1019B0000028ADD00B990029AADBC9086FF07E433F
:1019C000149D4FF0010E994228BF1946C5F3031329
:1019D0000EFA03F221FA03F303916161A261E3615C
:1019E000002B95D02646A44600274FF002081EAAD9
:1019F000C7F3460302EB830353F834AC07F001034B
:101A00001B01DA1D0EFA03F908FA02F2A2EB090231
:101A100002EA0A02DA401AD003F108090F330EFA7B
:101A200002F2216A08FA03F30EFA09FBCCF830201F
:101A30008A42A3EB0B0B0BEA0A0A2AFA09F98CF883
:101A40002C90A36A88BF2262934288BFA2620137AA
:101A50000CF1100C042FCAD1236A4FF0020C039A28
:101A60004FF0010E139F9A4224BFB2FBF3F1616263
:101A700007F00F0138BF01234FF0090201F1010106
:101A800038BF63624900336B33B3531C0EFA02F85C
:101A9000A2F105090CFA03F30EFA09FAA3EB080305
:101AA00002F1FF380CFA08F83B40A8EB0A08D340D3
:101AB00008EA070828FA09F87BD0012B7BD0022B13
:101AC0007BD0032B08BF4FF47A735FFA88F808FBCA
:101AD000033373634B43B36307321036252AD2D1E5
:101AE00015F0C04FC5F3417369D0012B69D0022BAB
:101AF0000CBF4FF47A634FF47A43C5F3046202FBE0
:101B00000333E3664B432367199B9E075CD0062390
:101B100084F8743015F4005F05F00F03C5F3042555
:101B200014BF40220822013305FB02255B00A56794
:101B30005D430A9B9F02E5677FF5EAAE0C9BC3F30A
:101B40000722C3F3421103F01F0384F8802084F8B6
:101B5000881084F88130002A3FF4DAAE189BC3F372
:101B6000025213F4401F84F883207FF4D1AEDE06C6
:101B700002D5042A7FF4CCAE03F40072002A14BF0D
:101B80000122002284F8872004D0DD0324D500231D
:101B900084F88930179B1A0722D5002384F88630F1
:101BA000702384F88530012384F88D301FB0BDE8A0
:101BB000F08F012389E7102387E7802385E710232F
:101BC0009BE74FF4807398E7590701D550239FE7AF
:101BD00013F0780F9ED09BE69903DBD50123D7E75E
:101BE0005B07E0D5012384F886300523D9E700BFE1
:101BF000DC68000830B58BB000240546806803928D
:101C00004FF00122059105A9CDE90624CDE908444C
:101C1000026852699047A8680121039B02680091FD
:101C2000214615692246A8470BB030BD13B50446BE
:101C3000A0680368DB6C98470028F9D10DF1070212
:101C400094F885102046FFF7D5FF94F886309DF86C
:101C500007001BB100F0010002B010BDC043C0F38B
:101C6000C010F9E730B54FF001238BB000240546D2
:101C700080688DF80F20059105A9CDE90634CDE9DE
:101C8000084403685B699847A86801220DF10F01B9
:101C9000036800941D692346A8470BB030BD0000BF
:101CA000F7B517460DF1070206461D46FFF7A2FFDE
:101CB00068B19DF8074039469DF82020304624EA57
:101CC00005042A4022438DF80720FFF7CBFF03B01D
:101CD000F0BD000030B54FF4807389B00024054694
:101CE0008068039103A9CDE90434CDE90644036873
:101CF0005B699847A86822462146036800941D69DD
:101D00002346A84709B030BD10B5044623682046D5
:101D1000DB6A98470028F9D110BD000010B590F893
:101D2000743004465BB1FFF7EFFF012394F87410A1
:101D3000204684F88E30BDE81040FFF7CBBF01206D
:101D400010BD000010B590F87430044653B1FFF791
:101D5000DBFF01232046042184F88E30BDE81040CB
:101D6000FFF7B8BF012010BDF0B590F883308BB0FD
:101D70000446042B50D100270DF10E0205218DF8E9
:101D80000E708DF80F70FFF735FF00282FD00DF182
:101D90000F0235212046FFF72DFF40B320461F4E8E
:101DA000FFF7BCFF2046FFF7AFFF05AD0FCE0FC515
:101DB000336805A99DF80E202B609DF80F30A068B0
:101DC00043F002038DF810208DF80F308DF811309C
:101DD00003685B699847A068022204A9036800971A
:101DE0001D693B46A84720B92046FFF7ABFF0020FE
:101DF00010E02046FFF7A6FF0DF10F023521204627
:101E0000FFF7F8FE0028F2D09DF80F309B07EED5C3
:101E1000012363600BB0F0BD0120FBE740680008C0
:101E20002DE9F341002304468068A36010B10368E4
:101E30005B6898470025264E264F0C2301A839469B
:101E40005FFA85F86B439A5900F072FA019BA0681B
:101E50000022A360019210B103685B689847019863
:101E600010B103685B689847A368E3B141F288301A
:101E700084F88C8002F076F82046FFF7D1FC1E2013
:101E800002F070F82046FFF7F9FC054688B994F88F
:101E90008C300C2210485343F158FFF737FB28468B
:101EA00002B0BDE8F0810135032DC6D10B4800F02A
:101EB0005BFB2046FFF758FF0C2294F88C30054658
:101EC0005343F15808B90648E7E70648E5E700BF7D
:101ED00084690008E4240020E46800085A690008C6
:101EE0000E690008386900082DE9F041044688B001
:101EF0000F461646FFF712FF2046FFF705FF0025A5
:101F0000C722A0684FF48073079503A9CDE9032386
:101F1000CDE9055503685B699847A0682A462946BC
:101F200003680095D3F810802B46C047054630B9AA
:101F30002046FFF707FF284608B0BDE8F081E36EB2
:101F40003B60236F3360F3E72DE9F041002588B053
:101F50001F4604460E460E9B00F1400CA8463D600D
:101F6000016B81B1A9420ED391420CD8B6FBF1FEB0
:101F700001FB1E6139B9416B90F82C800F9D1960EF
:101F8000816B2960154610306045E9D16DB3AB19FE
:101F90006269934229D82046FFF7C0FE2046FFF72A
:101FA000B3FE4FF41453A06803A9CDF80C80CDE91B
:101FB00004360026CDE9066603685B699847A06889
:101FC0003246314603680096D3F810803346C04746
:101FD000064620462EB9FFF7B5FE304608B0BDE8EC
:101FE000F081FFF7AFFE3D60F7E70026F5E7000060
:101FF0002DE9F0418669054688B00F46B342904608
:10200000B1FBF6FC06FB1C1C28BF3346A6EB0C0CF0
:1020100000269C45644628BF1C46FFF77FFE2846E5
:10202000FFF772FE0222A86803A9164B0597CDE9B7
:102030000323CDE9066603685B699847A8682246D2
:102040004146036800961F693346B847064628464E
:102050002EB9FFF777FE304608B0BDE8F081FFF7F4
:1020600071FE0E9B1C60AB6FAA696343B3FBF2F376
:102070000F9A1360EA6F109B5443AA69B4FBF2F401
:102080001C60E8E7002500012DE9F04FCE184369F8
:1020900089B004469E420F46914639D83D464FF4DA
:1020A0000458DFF878A0FFF72FFEAE4234D994F839
:1020B0008030A6EB050B94F8882003A90393002336
:1020C000BBF5806FA0680693636828BF4FF4806BF0
:1020D0000595012B14BF43465346012A049394F8F7
:1020E000813008BF03F1FF33079303685B699847AA
:1020F000A068A9EB07030268CDF800B02B44D2F822
:1021000010B000221146D84718B105F58065CCE71C
:10211000002009B0BDE8F08F0120FAE700ED0003D0
:10212000F0B5044689B00E46FFF7EEFD94F88750EF
:102130002DB194F889302BB1012B24D000252846ED
:1021400009B0F0BD94F880300393F02306934FF468
:10215000045304936368012B04BF1D4B04930023B5
:10216000059394F88130A06803A9079303685B691D
:102170009847A068314603689B69984705466420E4
:1021800001F0F0FEDBE720460027FFF7C7FD204601
:10219000FFF7BAFD08238122852120460097FFF72B
:1021A0007FFD054618B92046FFF7CCFDC7E794F838
:1021B000803006970393074B04936368012B04BF99
:1021C000054B04930023059394F88130013BCAE743
:1021D00000ED00030021001000ED0013014B024A46
:1021E0001A607047E4240020AC6A000830B50A4445
:1021F000084D91420DD011F8013B5840082340F39F
:102200000004013B2C4013F0FF0384EA5000F6D198
:10221000EFE730BD2083B8ED704700007047000045
:10222000002070470020704713B56C4600F114037E
:1022300084E8060094E8030083E8050002B010BDBE
:102240000020704713B56C4600F10C0384E80600CB
:1022500094E8030083E8050002B010BD0023C0E944
:102260000333704782B002AB03E9060002B0704747
:102270007047000000207047704700000020704742
:10228000002070470120704782B0002002A901E9B8
:102290000C0002B07047000000207047002070471B
:1022A000036B1A79034B53F832309B699868C0F37B
:1022B00040107047446A00080B6883634B684363AF
:1022C0008B68C363CB6803640B6943647047000089
:1022D00038B5036B0446154D1B7955F8330001F0F2
:1022E000BBFCD4E90B231B7955F8331002F1300302
:1022F0004968994218D000231363E26A5363D4E912
:102300000B12537C581E137C92681B0443EA002373
:1023100013438B63D4E90B131B79303155F8330029
:10232000BDE8384001F02CBC38BD00BF446A00084D
:10233000F8B51D4F05460E4611463868FFF732F9CD
:1023400078BB74683B7924B394F82C209A420BD064
:102350002468F8E70122B52100F010F973682360C2
:102360003B79746084F82C30482004F0DBF968B1C4
:1023700000220271C0E90322C0E90522027A42F07C
:1023800007020272094AC0E90B470260286028462A
:10239000F8BD402004F0C6F904460028DAD12C60CC
:1023A000F5E700232B60F2E7EC240020546A0008D4
:1023B000044B10B504460360406A08B104F0B0F95C
:1023C000204610BDF869000810B50446FFF7F0FF7D
:1023D000204604F0A3F9204610BD000008B519B14D
:1023E000FFF776FF012008BD036B1A79024B53F803
:1023F000320001F035FCF5E7446A00082DE9FF41A1
:10240000DDF828800546174603911FFA88F60293E7
:10241000FFF75EFF02ABBAB203A9E86A009600F0CC
:10242000C1F8044638B900212846FFF7D7FF2046F7
:1024300004B0BDE8F081AFB92B6B05F134011A7916
:10244000134B53F83200B8F1000F19D101F0A6FB7D
:1024500080F00104E4B23346E86ADDE9022100F0CD
:10246000C7F8E0E7029B83B92B6B3A46084805F1B1
:1024700034011C79039B50F8340001F0A5FBE7E719
:10248000029B424601F0B6FBE2E70024E3E700BF0F
:10249000446A000813B504460191FFF719FF019A39
:1024A000236B04F134011879054B53F8300001F027
:1024B000B7FB00212046FFF791FF012002B010BDBD
:1024C000446A000810B50446FFF702FF236B1A792F
:1024D000054B53F8320001F0B1FB00212046FFF715
:1024E0007DFF012010BD00BF446A0008064B01219A
:1024F000064A1A6000221A71054AC3E902124FF413
:102500008C721A82704700BFEC2400207B6900089F
:1025100000E1F50500F07EBA00B59BB0EFF309814C
:1025200068226846FFF720F8EFF30583014B9B6BA9
:10253000FEE700BF00ED00E008B5FFF7EDFF00008B
:1025400000B59BB0EFF3098168226846FFF70CF8ED
:10255000EFF30583014B5B6BFEE700BF00ED00E08E
:10256000FEE70000FEE700000FB408B5029801F096
:1025700085FCFEE702F0B0B902F088B938B5084B27
:1025800004461546017543600A21243002F042FAE0
:1025900004F128002A460A2102F03CFA204638BD00
:1025A000C06A0008F8B51E461B6805460C4617466B
:1025B0001BB9236863B9012408E0BDF8182031462F
:1025C000806A02F03FFA0028F3D100242046F8BDCB
:1025D00021463A46686A02F06BFA04460028EAD1BE
:1025E0003368002BF1D0A86A02F096FAEEE70000FB
:1025F00038B50D46114604461A4611B1806A02F0FC
:1026000049FA2DB12946606ABDE8384002F07CBA2B
:1026100038BD0000036800211B68184703790BB11F
:10262000002202711846704703685B681847000073
:1026300003791BB9012303711846704700207047C6
:102640007047000010B5044604F068F8204610BD3D
:10265000F0B500F10B0423460D46B1FBF2F102FB8D
:10266000115707F13006392EC8BF07F137069542DA
:1026700003F8016DF0D2421EE11A13F8015B9C428F
:1026800002F8015FF9D10844F0BD00002DE9F04FD8
:10269000804687B015464FF000090C4614F8013B00
:1026A000002B3BD0252B08D0D8F8002019464046F7
:1026B00009F10109D268904749E14B782D2B06BFFB
:1026C0008C1C01230023019323782B2B06BF01349C
:1026D0000127002794F800A0BAF1300F0CBF013495
:1026E0004FF0200A23782A2B1CD16178023455F848
:1026F00004BB2E2943D1217881B12A2921D0661C1F
:102700000020A1F130023446D2B2092A1DD80A2392
:1027100016F8011B03FB00200029F2D1484607B040
:10272000BDE8F08F4FF0000B14F8011B0029F5D025
:10273000A1F13002D2B2092ADBD80A2303FB0B2B0A
:10274000F2E76178023455F8040B01F0DF024C2AFD
:1027500017D121780029E1D0782904F101041FD88C
:10276000622900F2008158291AD84E2900F23081DE
:10277000442900F09180492900F08E8010E000206B
:10278000E3E7A1F141027829D2B209D862290BD836
:10279000582905D84E293BD8442978D0492976D0E4
:1027A0002E468DF80C1056E0A1F16306152EF7D8D1
:1027B0000FF2040C5CF826F0492800088F28000866
:1027C000A1270008A1270008A1270008A1270008C9
:1027D0008F280008A1270008A1270008A1270008CA
:1027E000A1270008A12700081F2900080D2A0008BA
:1027F000A1270008A12700085F280008A1270008DA
:10280000092A0008A1270008A12700080D2A0008AE
:10281000A1F14F02092AC3D801A050F822F000BF4D
:102820001F2900080D2A0008A1270008A127000879
:10283000A1270008A1270008092A0008A1270008ED
:10284000A12700080D2A00082E464FF0200A56F84E
:10285000042B8DF80C2003AD0DF10D002BE02E465E
:1028600047F6FF726A4B56F8045B002808BF104613
:10287000002D08BF1D462A462F18104612F8011BCE
:1028800011B1B91A0029F8DA4FF0200A13E02E46E8
:10289000192A56F8041B02D82E4656F8041B0029A4
:1028A00036DA2D2249428DF80C200DF10D000A2256
:1028B00003ADFFF7CDFE471B0199ABEB070323EAFE
:1028C000E372002945D1002BC2F1000B1EDD2978EF
:1028D0002D2901D02B290DD1BAF1300F0AD1D8F80A
:1028E00000304046019209F10109DB68013F984739
:1028F0000135019AD8F80030514640460192DB6814
:1029000098471BF1010B019AF4D191443B4615E025
:102910001FB12B228DF80C20C7E703A8C7E70822B8
:102920002E4603A856F8041BC2E7D8F800204046FC
:1029300015F8011BD26801939047019B013BF4D528
:10294000002FA8BFB9445D462DB9D944354621466C
:10295000A3E69346DAE7D8F8003051464046013DF9
:10296000DB689847F0E7A1F16302152A3FF618AF3C
:1029700001A353F822F000BF492800089928000855
:10298000A1270008A1270008A1270008A127000807
:1029900099280008A1270008A1270008A1270008FE
:1029A000A1270008A12700081F2900080D2A0008F8
:1029B000A1270008A12700085F280008A127000818
:1029C000092A0008A1270008A12700080D2A0008ED
:1029D000A1F14F02092A3FF6E3AE01A353F822F01A
:1029E0001F2900080D2A0008A1270008A1270008B8
:1029F000A1270008A1270008092A0008A12700082C
:102A0000A12700080D2A00080A2289E7102287E77B
:102A1000D86A0008F0B5054687B016461F460C4632
:102A200089B14A1E0023294601A800F05FF83A4602
:102A3000314601A8FFF72AFE049BA3423CBF0022B7
:102A4000EA5407B0F0BD0A46ECE70000D0E90223E3
:102A50009A421FBF4268D154C36801331ABFC36092
:102A600000206FF001007047D0E903239A421FBF96
:102A70004268D25C0133036114BF10466FF001005D
:102A80007047000003692BB1013B426803610020DD
:102A9000D15470476FF001007047000038B504460C
:102AA0000846D4E903315B1A934228BF13461D46FA
:102AB00063682A461944FEF757FD236928462B44CC
:102AC000236138BD38B50446D0E902301B1A934261
:102AD00028BF13461D4663682A461844FEF744FD86
:102AE000E36828462B44E36038BD000010B5C0E918
:102AF0000223034C0023C0E90041036110BD00BF65
:102B0000E06A00088A0710B504461DD50378042B37
:102B10001AD143681B682BB10522027098472378AD
:102B2000052B01D102232370302383F31188002168
:102B300004F1080001F030FA002383F31188E06902
:102B4000BDE8104002F05EB9CB0704D50248BDE8ED
:102B5000104001F093B910BDF86A000810B5044C9C
:102B6000204601F005F8034A0023C4E9062310BDFE
:102B7000042500200050005210B503780446012BB4
:102B800017D1104B984214D102460F49102002F081
:102B900005F90E4BE061D3F8D42042F48042C3F82B
:102BA000D420D3F8FC2042F48042C3F8FC20D3F8B0
:102BB000FC306268A36992685A60054A1A601B2259
:102BC000DA6010BD04250020052B000800440258DF
:102BD0001500020182691B2310B5D360D1E90030D2
:102BE00013F44C4406D19B011461D06103F44043BB
:102BF000536110BD0024184313F4406F1461CC6876
:102C0000D4615061F5D08B689361F2E730B5846987
:102C10001B25C069E5600068836104F12003C3617E
:102C200002234261013A03614223C3601623836297
:102C3000CB682261E361D1E90023134312F4406FB2
:102C4000636101D08B68A361C36843F00103C36073
:102C500030BD000030B5D0E90640006804F1200521
:102C60008561C36108234261013A036146230D690E
:102C7000C36016238362CB682261E361D1E900233C
:102C8000134312F4406F43EA854343F0806363616A
:102C900001D08B68A361C36843F00103C36030BDFA
:102CA0008069036823F0040310B5CC680360002337
:102CB0000361C4618361D1E900430969234343EAA5
:102CC000814343F04063436112B14FF010431360FE
:102CD00010BD000083691A6842F002021A601A6887
:102CE0009207FCD41A6842F004021A607047000090
:102CF0008269936810B5D3609B0704461DD503789D
:102D0000032B1AD143681B682BB105220270984728
:102D10002378052B01D102232370302383F31188FC
:102D2000002104F1080001F037F9002383F3118832
:102D3000E069BDE8104002F065B810BD0268436864
:102D40001143016003B1184770470000024A13683D
:102D500043F0C003136070470078004013B50E4C79
:102D6000204600F091FA04F1140000234FF40072A1
:102D70000A49009400F04EF9094B4FF400720949DA
:102D800004F13800009400F0C7F9074A074BC4E982
:102D9000172302B010BD00BF24250020902500207D
:102DA0004D2D0008902700200078004000E1F50537
:102DB000037C30B5244C002918BF0C46012B11D1DF
:102DC000224B98420ED1224BD3F8E82042F08042A9
:102DD000C3F8E820D3F8102142F08042C3F8102154
:102DE000D3F810312268036EC16D03EB5203846681
:102DF000B3FBF2F36268150442BF23F0070503F04A
:102E0000070343EA4503CB60A36843F040034B60EC
:102E1000E36843F001038B6042F4967343F00103CF
:102E20000B604FF0FF330B62510505D512F01022F5
:102E300005D0B2F1805F04D080F8643030BD7F23CC
:102E4000FAE73F23F8E700BF086B000824250020BD
:102E5000004402582DE9F047C66D05463768F4690D
:102E6000210734621AD014F0080118BF4FF48071A2
:102E7000E20748BF41F02001A3074FF0300348BFED
:102E800041F04001600748BF41F0800183F31188A1
:102E9000281DFFF753FF002383F31188E2050AD5AD
:102EA000302383F311884FF48061281DFFF746FF1C
:102EB000002383F311884FF030094FF0000A14F01B
:102EC000200838D13B0616D54FF0300905F1380AF5
:102ED000200610D589F31188504600F051F90028DA
:102EE00036DA0821281DFFF729FF27F08003336019
:102EF000002383F31188790614D5620612D5302396
:102F000083F31188D5E913239A4208D12B6C33B18E
:102F100027F040071021281DFFF710FF376000231E
:102F200083F31188E30618D5AA6E1369ABB1506913
:102F3000BDE8F047184789F31188736A284695F869
:102F40006410194000F0BAF98AF31188F469B6E701
:102F5000B06288F31188F469BAE7BDE8F087000031
:102F6000F8B51546826804460B46AA4200D2856829
:102F7000A1692669761AB5420BD218462A46FEF791
:102F8000F3FAA3692B44A3612846A3685B1BA360E3
:102F9000F8BD0CD9AF1B18463246FEF7E5FA3A46A3
:102FA000E1683044FEF7E0FAE3683B44EBE718469B
:102FB0002A46FEF7D9FAE368E5E700008368934202
:102FC000F7B50446154600D28568D4E90460361A80
:102FD000B5420BD22A46FEF7C7FA63692B446361F8
:102FE0002846A3685B1BA36003B0F0BD0DD9324631
:102FF000AF1B0191FEF7B8FA01993A46E0683144F7
:10300000FEF7B2FAE3683B44E9E72A46FEF7ACFA7A
:10301000E368E4E710B50A440024C361029B8460BE
:10302000C16002610362C0E90000C0E9051110BD82
:1030300008B5D0E90532934201D1826882B982682D
:10304000013282605A1C426119700021D0E90432B9
:103050009A4224BFC368436100F0B8FF002008BD56
:103060004FF0FF30FBE7000070B5302304460E46FA
:1030700083F31188A568A5B1A368A269013BA36089
:10308000531CA36115782269934224BFE368A361AE
:10309000E3690BB120469847002383F31188284643
:1030A00007E03146204600F081FF0028E2DA85F390
:1030B000118870BD2DE9F74F04460E461746984615
:1030C000D0F81C904FF0300A8AF311884FF0000BB3
:1030D000154665B12A4631462046FFF741FF0346B3
:1030E00060B94146204600F061FF0028F1D000237E
:1030F00083F31188781B03B0BDE8F08FB9F1000F9E
:1031000003D001902046C847019B8BF31188ED1A2C
:103110001E448AF31188DCE7C160C361009B8260B2
:103120000362C0E905111144C0E900000161704764
:10313000F8B504460D461646302383F31188A76878
:10314000A7B1A368013BA36063695A1C62611D704B
:10315000D4E904329A4224BFE3686361E3690BB1A6
:1031600020469847002080F3118807E0314620462A
:1031700000F01CFF0028E2DA87F31188F8BD000098
:10318000D0E9052310B59A4201D182687AB98268E4
:103190000021013282605A1C82611C7803699A42C4
:1031A00024BFC368836100F011FF204610BD4FF0BB
:1031B000FF30FBE72DE9F74F04460E4617469846C9
:1031C000D0F81C904FF0300A8AF311884FF0000BB2
:1031D000154665B12A4631462046FFF7EFFE034605
:1031E00060B94146204600F0E1FE0028F1D00023FE
:1031F00083F31188781B03B0BDE8F08FB9F1000F9D
:1032000003D001902046C847019B8BF31188ED1A2B
:103210001E448AF31188DCE70268436811430160A9
:1032200003B11847704700001430FFF743BF000098
:103230004FF0FF331430FFF73DBF00003830FFF789
:10324000B9BF00004FF0FF333830FFF7B3BF0000C5
:103250001430FFF709BF00004FF0FF311430FFF7C3
:1032600003BF00003830FFF763BF00004FF0FF32AC
:103270003830FFF75DBF0000012914BF6FF0130065
:1032800000207047FFF76ABD044B036000234360D2
:10329000C0E9023301230374704700BF206B0008AC
:1032A00010B53023044683F31188FFF781FD022314
:1032B0000020237480F3118810BD000038B5C36965
:1032C00004460D461BB904210844FFF7A5FF294613
:1032D00004F11400FFF7ACFE002806DA201D4FF4BD
:1032E0000061BDE83840FFF797BF38BD026843680A
:1032F0001143016003B118477047000013B5406BDC
:1033000000F58054D4F8A4381A681178042914D12F
:10331000017C022911D11979012312898B401342B2
:103320000BD101A94C3002F0CBFBD4F8A4480246E3
:10333000019B2179206800F0DFF902B010BD000088
:10334000143002F04DBB00004FF0FF33143002F098
:1033500047BB00004C3002F01FBC00004FF0FF33B1
:103360004C3002F019BC0000143002F01BBB00000E
:103370004FF0FF31143002F015BB00004C3002F06A
:10338000EBBB00004FF0FF324C3002F0E5BB000019
:103390000020704710B500F58054D4F8A4381A689E
:1033A0001178042917D1017C022914D159790123FC
:1033B00052898B4013420ED1143002F0ADFA02460E
:1033C00048B1D4F8A4484FF4407361792068BDE84F
:1033D000104000F07FB910BD406BFFF7DBBF00006D
:1033E000704700007FB5124B012504260446036098
:1033F0000023057400F1840243602946C0E90233CA
:103400000C4B0290143001934FF44073009602F07D
:103410005FFA094B04F69442294604F14C000294E9
:10342000CDE900634FF4407302F026FB04B070BD99
:10343000486B0008D9330008FD3200080A683023C1
:1034400083F311880B790B3342F823004B79133344
:1034500042F823008B7913B10B3342F8230000F5B7
:103460008053C3F8A41802230374002080F311884A
:103470007047000038B5037F044613B190F854300C
:10348000ABB90125201D0221FFF730FF04F1140024
:103490006FF00101257700F0A5FD04F14C0084F8E0
:1034A00054506FF00101BDE8384000F09BBD38BDBD
:1034B00010B5012104460430FFF718FF00232377DD
:1034C00084F8543010BD000038B50446002514308F
:1034D00002F016FA04F14C00257702F0E5FA201DFF
:1034E00084F854500121FFF701FF2046BDE8384021
:1034F000FFF750BF90F8803003F06003202B06D117
:1035000090F881200023212A03D81F2A06D8002002
:103510007047222AFBD1C0E91D3303E0034A42670A
:1035200007228267C3670120704700BF3422002052
:1035300037B500F58055D5F8A4381A6811780429F4
:103540001AD1017C022917D11979012312898B40E4
:10355000134211D100F14C04204602F065FB58B132
:1035600001A9204602F0ACFAD5F8A4480246019B16
:103570002179206800F0C0F803B030BD01F10B03E1
:10358000F0B550F8236085B004460D46FEB13023F7
:1035900083F3118804EB8507301D0821FFF7A6FE91
:1035A000FB6806F14C005B691B681BB1019002F0DF
:1035B00095FA019803A902F083FA024648B1039BE9
:1035C0002946204600F098F8002383F3118805B0BF
:1035D000F0BDFB685A691268002AF5D01B8A013BCE
:1035E0001340F1D104F18002EAE70000133138B54D
:1035F00050F82140ECB1302383F3118804F5805357
:10360000D3F8A4281368527903EB8203DB689B6923
:103610005D6845B104216018FFF768FE294604F192
:10362000140002F083F92046FFF7B4FE002383F371
:10363000118838BD7047000001F03ABC01234022D8
:10364000002110B5044600F8303BFDF7BFFF002312
:10365000C4E9013310BD000010B53023044683F3E4
:1036600011882422416000210C30FDF7AFFF204675
:1036700001F040FC02230020237080F3118810BD6C
:1036800070B500EB8103054650690E461446DA60BA
:1036900018B110220021FDF799FFA06918B110227E
:1036A0000021FDF793FF31462846BDE8704001F048
:1036B00027BD000083682022002103F0011310B50C
:1036C000044683601030FDF781FF2046BDE81040BE
:1036D00001F0A2BDF0B4012500EB810447898D40C3
:1036E000E4683D43A469458123600023A2606360D0
:1036F000F0BC01F0BFBD0000F0B4012500EB810477
:1037000007898D40E4683D43646905812360002397
:10371000A2606360F0BC01F035BE000070B502230A
:1037200000250446242203702946C0F888500C3036
:1037300040F8045CFDF74AFF204684F8705001F021
:1037400073FC63681B6823B129462046BDE87040BE
:10375000184770BD0378052B10B504460AD080F8D1
:103760008C300523037043681B680BB10421984714
:103770000023A36010BD00000178052906D190F850
:103780008C20436802701B6803B118477047000023
:1037900070B590F87030044613B1002380F8703093
:1037A00004F18002204601F05BFD63689B68B3B9B9
:1037B00094F8803013F0600535D00021204602F0E7
:1037C0004DF80021204602F03DF863681B6813B1F4
:1037D000062120469847062384F8703070BD2046A5
:1037E00098470028E4D0B4F88630A26F9A4288BF88
:1037F000A36794F98030A56F002B4FF0300380F25F
:103800000381002D00F0F280092284F8702083F3F8
:10381000118800212046D4E91D23FFF76DFF002306
:1038200083F31188DAE794F8812003F07F0343EAF9
:10383000022340F20232934200F0C58021D8B3F552
:10384000807F48D00DD8012B3FD0022B00F0938011
:10385000002BB2D104F1880262670222A267E367FB
:10386000C1E7B3F5817F00F09B80B3F5407FA4D121
:1038700094F88230012BA0D1B4F8883043F00203D1
:1038800032E0B3F5006F4DD017D8B3F5A06F31D04B
:10389000A3F5C063012B90D86368204694F882207A
:1038A0005E6894F88310B4F88430B047002884D060
:1038B000436863670368A3671AE0B3F5106F36D0F7
:1038C00040F6024293427FF478AF5C4B6367022379
:1038D000A3670023C3E794F88230012B7FF46DAF18
:1038E000B4F8883023F00203A4F88830C4E91D55E9
:1038F000E56778E7B4F88030B3F5A06F0ED194F89F
:103900008230204684F88A3001F0ECFB63681B6843
:1039100013B1012120469847032323700023C4E9F3
:103920001D339CE704F18B0363670123C3E723780E
:10393000042B10D1302383F311882046FFF7BAFE01
:1039400085F311880321636884F88B5021701B680C
:103950000BB12046984794F88230002BDED084F8D3
:103960008B300423237063681B68002BD6D00221A0
:1039700020469847D2E794F8843020461D0603F08D
:103980000F010AD501F05EFC012804D002287FF463
:1039900014AF2B4B9AE72B4B98E701F045FCF3E76C
:1039A00094F88230002B7FF408AF94F8843013F041
:1039B0000F01B3D01A06204602D501F067FFADE72C
:1039C00001F058FFAAE794F88230002B7FF4F5AE9F
:1039D00094F8843013F00F01A0D01B06204602D5C6
:1039E00001F03CFF9AE701F02DFF97E7142284F8DD
:1039F000702083F311882B462A4629462046FFF77C
:103A000069FE85F31188E9E65DB1152284F870201E
:103A100083F3118800212046D4E91D23FFF75AFEC5
:103A2000FDE60B2284F8702083F311882B462A468A
:103A300029462046FFF760FEE3E700BF786B0008E9
:103A4000706B0008746B000838B590F8703004464D
:103A5000002B3ED0063BDAB20F2A34D80F2B32D8D7
:103A6000DFE803F037313108223231313131313181
:103A700031313737856FB0F886309D4214D2C36834
:103A80001B8AB5FBF3F203FB12556DB9302383F3A8
:103A900011882B462A462946FFF72EFE85F311880A
:103AA0000A2384F870300EE0142384F87030302339
:103AB00083F31188002320461A461946FFF70AFEB1
:103AC000002383F3118838BDC36F03B198470023E7
:103AD000E7E70021204601F0C1FE0021204601F069
:103AE000B1FE63681B6813B1062120469847062380
:103AF000D7E7000010B590F870300446142B29D099
:103B000017D8062B05D001D81BB110BD093B022BDD
:103B1000FBD80021204601F0A1FE0021204601F043
:103B200091FE63681B6813B106212046984706235F
:103B300019E0152BE9D10B2380F87030302383F383
:103B4000118800231A461946FFF7D6FD002383F398
:103B50001188DAE7C3689B695B68002BD5D1C36F16
:103B600003B19847002384F87030CEE7FEF7F6BF24
:103B7000012100230170C0E901330C3000F028B9A5
:103B800010B53023044683F311884160FEF7F4FF3B
:103B900002230020237080F3118810BD10B530235C
:103BA000044683F31188032304F8083BFFF712F857
:103BB0004FF0FF31204600F0E1F9002383F3118834
:103BC000C01A18BF012010BD38B50446302585F352
:103BD0001188032504F8085BFFF718F84FF0FF3150
:103BE000204600F0CBF9002383F31188C01A18BFD8
:103BF000012038BD38B50446302585F311880425E9
:103C000004F8085BFFF726F84FF0FF31204600F07C
:103C1000B5F9002383F31188C01A18BF012038BDFD
:103C200010B53023044683F31188FFF739F80623D3
:103C30002370002383F3118810BD000010B53023DA
:103C4000044683F31188FFF745F80223237000230D
:103C500083F3118810BD00000C3000F0D5B80000CF
:103C60000C3000F0DBB800000023826803750369A4
:103C70001B6899689142FBD25A68036042601060E9
:103C80005860704700238268037503691B68996850
:103C90009142FBD85A6803604260106058607047D8
:103CA00008B50846302383F311880A7D0023052ACE
:103CB00006D8DFE802F00B050503120E82691360D7
:103CC0004FF0FF338361FFF7CFFF002383F31188A9
:103CD00008BD8269936801339360D0E900321360B4
:103CE0005A60EDE7FFF7C0BF054BD9680875186843
:103CF000026853601A600122D8600275FCF70CBD9F
:103D0000902900200C4B30B5DD684B1C87B0044671
:103D10000FD02B46094A684600F0F8F92046FFF715
:103D2000E3FF009B13B1684600F0FAF9A86907B0F9
:103D300030BDFFF7D9FFF9E790290020A13C00082A
:103D400038B50C4D04468161EB6881689A689142F0
:103D500003D8BDE83840FFF787BF1846FFF792FF4A
:103D600001230146EC6020462375BDE83840FCF78E
:103D7000D3BC00BF90290020044B1A68DB68906810
:103D80009B68984294BF0020012070479029002032
:103D9000084B10B51C68D868226853601A6001226D
:103DA000DC602275FFF76EFF01462046BDE810403B
:103DB000FCF7B2BC90290020044B1A68DB689268BB
:103DC0009B689A4201D9FFF7E3BF70479029002012
:103DD000C0E90000816070478368013B002B10B58B
:103DE00083600CDA074BDC684368A0612060636085
:103DF0001C6044600520FFF777FFA06910BD00201C
:103E0000FCE700BF9029002008B5302383F3118818
:103E1000FFF7E2FF002383F3118808BD08B53023C4
:103E200083F3118883680133002B836007DC036808
:103E300000211A68026050601846FFF781FF0023D6
:103E400083F3118808BD000038B50123084C002514
:103E50002370656001F024FF01F04AFF0549064820
:103E600002F01EF80223237085F3118838BD00BFCD
:103E7000F82B0020806B00089029002008B572B64E
:103E8000044B186500F0F4FC00F0C2FD024B032265
:103E90001A70FEE790290020F82B002000F076B978
:103EA000EFF3118020B9EFF30583302282F31188FC
:103EB0007047000010B530B9EFF30584C4F308046F
:103EC00014B180F3118810BDFFF776FF84F31188D9
:103ED000F9E70000034A516853685B1A9842FBD81F
:103EE000704700BF001000E08B60022308610846A5
:103EF0008B8270478368A3F1840243F8142C026913
:103F000043F8442C426943F8402C094A43F8242CD6
:103F1000C268A3F1200043F8182C022203F80C2CED
:103F2000002203F80B2C034A43F8102C704700BF03
:103F3000310700089029002008B5FFF7DBFFBDE836
:103F40000840FFF7CFBE0000024BDB6898610F20EE
:103F5000FFF7CABE90290020302383F31188FFF7B2
:103F6000F3BF000008B50146302383F31188082011
:103F7000FFF7C8FE002383F3118808BD054BDB68FB
:103F800021B1036098610320FFF7BCBE4FF0FF3002
:103F9000704700BF9029002003682BB10022026007
:103FA00018469961FFF79EBE70470000064BDB681C
:103FB00039B1426818605A60136043600420FFF70B
:103FC000A1BE4FF0FF30704790290020036898424F
:103FD00006D01A680260506018469961FFF782BEE9
:103FE0007047000038B504460D462068844200D171
:103FF00038BD036823605C608561FFF773FEF4E7FA
:10400000036810B59C68A2420CD85C688A600B609B
:104010004C602160596099688A1A9A604FF0FF33AA
:10402000836010BD121B1B68ECE700000A2938BF33
:104030000A2170B504460D460A26601901F02AFED1
:1040400001F012FE041BA54203D8751C04462E463F
:10405000F3E70A2E04D90120BDE8704001F060BFEB
:1040600070BD0000F8B5144B0D460A2A4FF00A0740
:10407000D96103F11001826038BF0A2241601969D9
:104080001446016048601861A81801F0F3FD01F0C2
:10409000EBFD431B0646A34206D37C1C281927468A
:1040A000354601F0F7FDF2E70A2F04D90120BDE8FB
:1040B000F84001F035BFF8BD90290020F8B506465C
:1040C0000D4601F0D1FD0F4A134653F8107F9F4271
:1040D00006D12A4601463046BDE8F840FFF7C2BF88
:1040E000D169BB68441A2C1928BF2C46A34202D9B7
:1040F0002946FFF79BFF224631460348BDE8F840BA
:10410000FFF77EBF90290020A0290020C0E90323EB
:10411000002310B45DF8044B4361FFF7CFBF0000EC
:1041200010B5194C236998420DD08168D0E900324E
:1041300013605A609A680A449A60002303604FF043
:10414000FF33A36110BD0268234643F8102F53606C
:104150000022026022699A4203D1BDE8104001F0BA
:1041600093BD936881680B44936001F07DFD2269E3
:10417000E1699268441AA242E4D91144BDE81040B2
:10418000091AFFF753BF00BF902900202DE9F0471F
:10419000DFF8BC8008F110072C4ED8F8105001F061
:1041A00063FDD8F81C40AA68031B9A423ED8144409
:1041B0004FF00009D5E90032C8F81C4013605A607E
:1041C000C5F80090D8F81030B34201D101F05CFD81
:1041D00089F31188D5E9033128469847302383F3C2
:1041E00011886B69002BD8D001F03EFD6A69A0EB05
:1041F000040982464A450DD2022001F091FE0022B8
:10420000D8F81030B34208D151462846BDE8F047EF
:10421000FFF728BF121A2244F2E712EB09092946D8
:10422000384638BF4A46FFF7EBFEB5E7D8F81030FE
:10423000B34208D01444C8F81C00211AA960BDE894
:10424000F047FFF7F3BEBDE8F08700BFA0290020CC
:104250009029002000207047FEE700007047000012
:104260004FF0FF307047000002290CD0032904D022
:104270000129074818BF00207047032A05D80548C0
:1042800000EBC2007047044870470020704700BF31
:10429000586C0008442200200C6C000870B59AB0DD
:1042A00005460846144601A900F0C2F801A8FDF72A
:1042B00085F9431C0022C6B25B001046C5E90034F4
:1042C00023700323023404F8013C01ABD1B2023461
:1042D0008E4201D81AB070BD13F8011B013204F8E8
:1042E000010C04F8021CF1E708B5302383F31188B0
:1042F0000348FFF71DF9002383F3118808BD00BFB1
:10430000002C002090F8803003F01F02012A07D112
:1043100090F881200B2A03D10023C0E91D3315E05A
:1043200003F06003202B08D1B0F884302BB990F84B
:104330008120212A03D81F2A04D8FFF7DBB8222ABC
:10434000EBD0FAE7034A426707228267C36701207E
:10435000704700BF3B22002007B5052917D8DFE8CA
:1043600001F0191603191920302383F31188104A1C
:1043700001210190FFF784F9019802210D4AFFF70E
:104380007FF90D48FFF7A0F8002383F3118803B0ED
:104390005DF804FB302383F311880748FFF76AF8C0
:1043A000F2E7302383F311880348FFF781F8EBE746
:1043B000AC6B0008D06B0008002C002038B50C4D09
:1043C0000C4C2A460C4904F10800FFF767FF05F181
:1043D000CA0204F110000949FFF760FF05F5CA722F
:1043E00004F118000649BDE83840FFF757BF00BF89
:1043F000D8440020442200208C6B0008966B0008F3
:10440000A16B000870B5044608460D46FDF7D6F8C6
:10441000C6B22046013403780BB9184670BD324647
:104420002946FDF7ABF80028F3D10120F6E700009C
:104430002DE9F84F05460C46FDF7C0F82C49C6B2E9
:104440002846FFF7DFFF08B10336F6B229492846B0
:10445000FFF7D8FF08B11036F6B2632E0DD8DFF89B
:104460009080DFF89090244FDFF894A0DFF894B0AC
:104470002E7846B92670BDE8F88F29462046BDE85B
:10448000F84F02F0D3B9252E2ED1072241462846F7
:10449000FDF774F870B9DBF8003007350A3444F8DA
:1044A0000A3CDBF8043044F8063CBBF8083024F83A
:1044B000023CDDE7082249462846FDF75FF898B937
:1044C000A21C0E4B197802320909C95D02F8041CBE
:1044D00013F8011B01F00F015345C95D02F8031CDD
:1044E000F0D118340835C3E7013504F8016BBFE794
:1044F000786C0008A16B00088B6C000800E8F11FC5
:104500000CE8F11F806C0008BFF34F8F024A13695B
:104510005B07FCD1704700BF0020005208B5074B75
:104520001B7853B9FFF7F0FF054BDA68D20704D5C3
:10453000044A5A6002F188325A6008BD36470020AA
:1045400000200052230167454FF00063054A1968B7
:10455000013104D104339342F9D101207047002086
:10456000704700BF0000020808B5094B1B786BB903
:1045700008490B695B0703D5CB6843F04003CB6068
:10458000FFF7C2FFCB6843F00103CB6008BD00BF5B
:1045900036470020002000524FF4003070470000E2
:1045A0000120704708B9FFF7CFBF00207047000017
:1045B00008B508BB1149FFF7A7FFFFF7AFFF4FF0A2
:1045C000FF334B610B61FFF79FFF2423CB60CB6868
:1045D00043F08003CB600B695B07FCD44FF40031E0
:1045E0004FF00060FFF790FF00F0EEF9FFF7BCFF1F
:1045F000BDE80840FFF7A8BF002008BD002000521A
:104600002DE9F84340EA02030C4605461146DE0652
:1046100002D00020BDE8F88321F01F01224F4FF0A7
:10462000FF38FFF77BFF6618B44203D10120FFF784
:104630009BFFEFE720222946204602F0A3F810B99D
:1046400020352034F0E72B4605F120021968481C7C
:10465000DFD104339342F9D1FFF756FF7961FB684C
:10466000291B04F11C0243F00203FB60231F38697D
:1046700010F00509FBD153F8040F9A42C850F6D147
:10468000BFF34F8FFFF740FFC7F81480FB6820226D
:104690002146284623F00203FB6002F073F800284D
:1046A000CED04846C3E700BF00200052084908B5F5
:1046B0000B7828B11BB9FFF731FF01230B7008BD40
:1046C000002BFCD00870BDE80840FFF74DBF00BFCD
:1046D000364700202DE9F04F0D4685B0814658B190
:1046E00011F00D0614BF2022082211F008030193D7
:1046F00004D0431E03426AD0002435E0002E37D098
:1047000009F11F0121F01F094FF00108324F05F098
:104710000403DFF8D0A005EA080BBBF1000F32D08C
:104720007869C0072FD408F101080C37B8F1060FDB
:10473000F3D19EB9294D4946A819019201F0FAFA20
:10474000044600283AD11836019A782EF3D149460A
:1047500001F0F0FA0446002830D1019A4946204879
:1047600001F0E8FA044668BB204605B0BDE8F08FCA
:104770000029C9D101462846029201F0DBFA04461D
:10478000E0B9029AC0E713B178694107CBD5AC070D
:1047900002D578698007C6D5019911B178690107FA
:1047A000C1D51820494600FB08A0CDE9022301F03D
:1047B000C1FA0446DDE902230028B4D04A460021AC
:1047C000204601E04A460021FCF700FFCCE7024604
:1047D000002E95D198E700BF9C6C00086847002028
:1047E00038470020504700200021FFF773BF00002A
:1047F0000121FFF76FBF0000F8B5144D0124182701
:10480000134E40F2FF3200210120FCF7DFFE07FBD0
:10481000046001342A6955F80C1F01F077FA062C60
:10482000F5D137254FF4C0542046FFF7E1FF01468C
:1048300028B122460748BDE8F84001F067BAC4EB4A
:10484000C404013D4FEAD404EED1F8BD9C6C0008CD
:1048500050470020384700200421FFF73BBF0000ED
:104860004843FFF7C1BF000008B101F0D5BA704757
:1048700038B5054D00240334696855F80C0B00F079
:10488000B5F8122CF7D138BD9C6C000870B5104EED
:1048900082B0FFF705FB054601F0E6F932680346F2
:1048A0009042336037BF0B4A0A495168146836BFDB
:1048B0000131D1E9004151600419284641F100015C
:1048C0000191FFF7F7FA2046019902B070BD00BFD1
:1048D000E0470020E847002070B5124E82B0FFF795
:1048E000DFFA054601F0C0F93268034690423360B2
:1048F00037BF0D4A0C495168146836BF0131D1E900
:10490000004151600419284641F100010191FFF76F
:10491000D1FA4FF47A72002320460199FBF7E8FCA4
:1049200002B070BDE0470020E84700200244074B7A
:10493000D2B210B5904200D110BD441C00B253F861
:10494000200041F8040BE0B2F4E700BF50400058EB
:104950000E4B30B51C6F240405D41C6F1C671C6FF4
:1049600044F400441C670A4C02442368D2B243F466
:1049700080732360074B904200D130BD441C51F836
:10498000045B00B243F82050E0B2F4E70044025860
:10499000004802585040005807B5012201A90020E4
:1049A000FFF7C4FF019803B05DF804FB13B504469C
:1049B000FFF7F2FFA04205D0012201A900200194D7
:1049C000FFF7C6FF02B010BD0144BFF34F8F064B87
:1049D000884204D3BFF34F8FBFF36F8F7047C3F884
:1049E0005C022030F4E700BF00ED00E00144BFF3BB
:1049F0004F8F064B884204D3BFF34F8FBFF36F8FA7
:104A00007047C3F870022030F4E700BF00ED00E00B
:104A10007047000070B5054616460C46012010216F
:104A2000FFF71EFF286046733CB1204636B1FFF702
:104A300013FF2B68186000B19C6070BDFFF7D8FEB3
:104A4000F7E7000070B50E461546044600B30B6844
:104A500043608368934210D213B10068FFF704FFEC
:104A6000637B28462BB1FFF7F7FE206020B9A060DA
:104A700070BDFFF7BDFEF8E7A560206805F11F01D6
:104A8000306021F01F01FFF79FFF01202073EFE747
:104A90000120EDE710B5044640B10068884205D119
:104AA000606808B1FCF760FD0023237310BD0000AF
:104AB00070B50E461546044620B383689A4210D955
:104AC00013B10068FFF7D0FE637B28462BB1FFF7D8
:104AD000C3FE206020B9A06070BDFFF789FEF8E733
:104AE000A560316819B12A462068FCF73DFD2068B1
:104AF00005F11F01306021F01F01FFF777FF012052
:104B00002073E9E70120E7E720B103688B4204BF87
:104B1000002303737047000008B10023037370473C
:104B2000034B1A681AB9034AD2F8D0241A607047A6
:104B3000F04700200040025808B5FFF7F1FF024B94
:104B40001868C0F3806008BDF047002070B5BFF35F
:104B50004F8FBFF36F8F1A4A0021C2F85012BFF374
:104B60004F8FBFF36F8F536943F400335361BFF32B
:104B70004F8FBFF36F8FC2F88410BFF34F8FD2F8FF
:104B8000803043F6E074C3F3C900C3F34E335B01D6
:104B900003EA0406014646EA81750139C2F860520B
:104BA000F9D2203B13F1200FF2D1BFF34F8F53699D
:104BB00043F480335361BFF34F8FBFF36F8F70BDEA
:104BC00000ED00E0FEE70000214B2248224A70B5CC
:104BD000904237D3214BC11EDA1C121A22F0030275
:104BE0008B4238BF00220021FCF7F0FC1C4A002356
:104BF000C2F88430BFF34F8FD2F8803043F6E074B0
:104C0000C3F3C900C3F34E335B0103EA0406014654
:104C100046EA81750139C2F86C52F9D2203B13F192
:104C2000200FF2D1BFF34F8FBFF36F8FBFF34F8FC2
:104C3000BFF36F8F0023C2F85032BFF34F8FBFF323
:104C40006F8F70BD53F8041B40F8041BC0E700BF12
:104C5000706F0008B04A0020B04A0020B04A00201F
:104C600000ED00E003681A6899685A6043681BB158
:104C700042EA014180681847704700004FF0A443A2
:104C800010B51C68E00702D52848FFF7EBFFA10725
:104C900002D52748FFF7E6FF620702D52548FFF750
:104CA000E1FF230702D52448FFF7DCFFE00602D529
:104CB0002248FFF7D7FFA10602D52148FFF7D2FF10
:104CC000620602D51F48FFF7CDFF230602D51E4816
:104CD000FFF7C8FFE00502D51C48FFF7C3FFA10599
:104CE00002D51B48FFF7BEFF620502D51948FFF742
:104CF000B9FF230502D51848FFF7B4FFE00402D539
:104D00001648FFF7AFFFA10402D51548FFF7AAFF29
:104D1000620402D51348FFF7A5FF230402D5124809
:104D2000FFF7A0FFBDE8104001F0ECB9F847002004
:104D300004480020104800201C480020284800207B
:104D400034480020404800204C48002058480020AB
:104D500064480020704800207C48002088480020DB
:104D600094480020A0480020AC48002030B5094BF2
:104D70000021094C10200725196054F8042B013834
:104D8000C3E90121D16003F10C0311615560F4D135
:104D900030BD00BFF4470020E46C00080F28F0B5D8
:104DA0000AD9102806D10F230020144C01272568AA
:104DB000984203D900201DE00346F6E707FA00F603
:104DC000354218D10C23354343432560181D234435
:104DD000C3E902120A4B2044D3F8D42042F0010266
:104DE000C3F8D420D3F8FC2042F00102C3F8FC2021
:104DF000D3F8FC30F0BD0130DAE700BFF447002003
:104E0000004402580368D968DA68C90722F03F02F3
:104E1000DA6002D51A689207FCD507225A607047FB
:104E2000074BD3F8D81021EA0001C3F8D810D3F803
:104E3000002122EA0002C3F80021D3F800317047B4
:104E40000044025870B5D0E9244300224FF0FF35EA
:104E50009E6804EB42135101D3F80009002805DADB
:104E6000D3F8000940F08040C3F80009D3F8000BE4
:104E7000002805DAD3F8000B40F08040C3F8000B9F
:104E8000013263189642C3F80859C3F8085BE0D2B0
:104E90004FF00113C4F81C3870BD0000890141F0C7
:104EA0002001016103699B06FCD41220FFF712B8B0
:104EB00010B50A4C2046FEF7C1FB094BC4F89030F0
:104EC000084BC4F89430084C2046FEF7B7FB074B5C
:104ED000C4F89030064BC4F8943010BDB848002098
:104EE00000000840486D00085449002000000440BC
:104EF000546D000870B503780546012B5CD1434B17
:104F0000D0F89040984258D1414B0E216520D3F8FB
:104F1000D82042F00062C3F8D820D3F8002142F034
:104F20000062C3F80021D3F80021D3F8802042F0BA
:104F30000062C3F88020D3F8802022F00062C3F81A
:104F40008020D3F8803000F0ADFC324BE360324B70
:104F5000C4F800380023D5F89060C4F8003EC023A0
:104F600023604FF40413A3633369002BFCDA01239D
:104F70000C203361FEF7AEFF3369DB07FCD412204F
:104F8000FEF7A8FF3369002BFCDA00262846A6604E
:104F9000FFF758FF6B68C4F81068DB68C4F8146842
:104FA000C4F81C6883BB1D4BA3614FF0FF336361E2
:104FB000A36843F00103A36070BD194B9842C9D1A7
:104FC000134B4FF08060D3F8D82042F00072C3F842
:104FD000D820D3F8002142F00072C3F80021D3F8A2
:104FE0000021D3F8802042F00072C3F88020D3F86B
:104FF000802022F00072C3F88020D3F88030FFF7C1
:105000000FFF0E214D209EE7064BCDE7B84800204C
:10501000004402584014004003002002003C30C00D
:1050200054490020083C30C0F8B5D0F890400546FF
:1050300000214FF000662046FFF730FFD5F89410AE
:1050400000234FF001128F684FF0FF30C4F834385E
:10505000C4F81C2804EB431201339F42C2F80069D4
:10506000C2F8006BC2F80809C2F8080BF2D20B684C
:10507000D5F89020C5F89830636210231361166943
:1050800016F01006FBD11220FEF724FFD4F80038EA
:1050900023F4FE63C4F80038A36943F4402343F0CB
:1050A0001003A3610923C4F81038C4F814380B4B5B
:1050B000EB604FF0C043C4F8103B094BC4F8003B11
:1050C000C4F81069C4F80039D5F8983003F110021B
:1050D00043F48013C5F89820A362F8BD246D00083E
:1050E00040800010D0F8902090F88A10D2F8003854
:1050F00023F4FE6343EA0113C2F80038704700004E
:105100002DE9F84300EB8103D0F890500C4680461F
:10511000DA680FFA81F94801166806F00306731E73
:10512000022B05EB41134FF0000194BFB604384E3B
:10513000C3F8101B4FF0010104F1100398BF06F1F2
:10514000805601FA03F3916998BF06F500460029DD
:105150003AD0578A04F15801374349016F50D5F8C6
:105160001C180B430021C5F81C382B180127C3F865
:105170001019A7405369611E9BB3138A928B9B0839
:10518000012A88BF5343D8F89820981842EA03436D
:1051900001F140022146C8F89800284605EB82023A
:1051A0005360FFF77BFE08EB8900C3681B8A43EA64
:1051B000845348341E4364012E51D5F81C381F43D4
:1051C000C5F81C78BDE8F88305EB4917D7F8001B34
:1051D00021F40041C7F8001BD5F81C1821EA03038D
:1051E000C0E704F13F030B4A2846214605EB830341
:1051F0005A60FFF753FE05EB4910D0F8003923F44D
:105200000043C0F80039D5F81C3823EA0707D7E770
:105210000080001000040002D0F894201268C0F84A
:105220009820FFF70FBE00005831D0F890304901A8
:105230005B5813F4004004D013F4001F0CBF02208D
:10524000012070474831D0F8903049015B5813F481
:10525000004004D013F4001F0CBF0220012070474F
:1052600000EB8101CB68196A0B6813604B685360CF
:105270007047000000EB810330B5DD68AA69136850
:10528000D36019B9402B84BF402313606B8A146824
:10529000D0F890201C4402EB4110013C09B2B4FB51
:1052A000F3F46343033323F0030343EAC44343F0BB
:1052B000C043C0F8103B2B6803F00303012B0ED151
:1052C000D2F8083802EB411013F4807FD0F8003B8D
:1052D00014BF43F0805343F00053C0F8003B02EB8F
:1052E0004112D2F8003B43F00443C2F8003B30BD0A
:1052F0002DE9F041D0F8906005460C4606EB4113CD
:10530000D3F8087B3A07C3F8087B08D5D6F81438D9
:105310001B0704D500EB8103DB685B689847FA073D
:105320001FD5D6F81438DB071BD505EB8403D968E5
:10533000CCB98B69488A5A68B2FBF0F600FB16229A
:105340008AB91868DA6890420DD2121AC3E90024AB
:10535000302383F3118821462846FFF78BFF84F31F
:105360001188BDE8F081012303FA04F26B8923EA76
:1053700002036B81CB68002BF3D021462846BDE8A1
:10538000F041184700EB81034A0170B5DD68D0F8A1
:1053900090306C692668E66056BB1A444FF40020D2
:1053A000C2F810092A6802F00302012A0AB20ED1DB
:1053B000D3F8080803EB421410F4807FD4F80009F6
:1053C00014BF40F0805040F00050C4F8000903EBD7
:1053D0004212D2F8000940F00440C2F8000901224C
:1053E000D3F8340802FA01F10143C3F8341870BD50
:1053F00019B9402E84BF4020206020681A442E8AAC
:105400008419013CB4FBF6F440EAC44040F000507B
:10541000C6E700002DE9F843D0F8906005460C4639
:105420004F0106EB4113D3F8088918F0010FC3F8B8
:1054300008891CD0D6F81038DB0718D500EB81039B
:10544000D3F80CC0DCF81430D3F800E0DA689645E5
:1054500030D2A2EB0E024FF000091A60C3F804909C
:10546000302383F31188FFF78DFF89F3118818F03B
:10547000800F1DD0D6F834380126A640334217D00D
:1054800005EB84030134D5F89050D3F80CC0E4B296
:105490002F44DCF8142005EB0434D2F800E0516806
:1054A000714514D3D5F8343823EA0606C5F83468B4
:1054B000BDE8F883012303FA01F2038923EA02031A
:1054C0000381DCF80830002BD1D09847CFE7AEEB52
:1054D0000103BCF81000834228BF0346D7F818091F
:1054E00080B2B3EB800FE3D89068A0F1040959F8BB
:1054F000048FC4F80080A0EB09089844B8F1040FA9
:10550000F5D818440B4490605360C8E72DE9F84F74
:10551000D0F8905004466E69AB691E4016F480586E
:105520006E6103D0BDE8F84FFEF7F8B8002E12DA2E
:10553000D5F8003E9B0705D0D5F8003E23F00303C5
:10554000C5F8003ED5F80438204623F00103C5F81D
:105550000438FEF711F9370505D52046FFF772FC30
:105560002046FEF7F7F8B0040CD5D5F8083813F04C
:10557000060FEB6823F470530CBF43F4105343F44D
:10558000A053EB6031071BD56368DB681BB9AB69BF
:1055900023F00803AB612378052B0CD1D5F8003E2E
:1055A0009A0705D0D5F8003E23F00303C5F8003E66
:1055B0002046FEF7E1F86368DB680BB120469847A8
:1055C000F30200F1BA80B70226D5D4F890900027F4
:1055D0004FF0010A09EB4712D2F8003B03F44023D5
:1055E000B3F5802F11D1D2F8003B002B0DDA628980
:1055F0000AFA07F322EA0303638104EB8703DB68FB
:10560000DB6813B13946204698470137D4F8943007
:10561000FFB29B689F42DDD9F00619D5D4F89000FF
:10562000026AC2F30A1702F00F0302F4F012B2F595
:10563000802F00F0CA80B2F5402F09D104EB83031C
:10564000002200F58050DB681B6A974240F0B08072
:105650003003D5F8185835D5E90303D50021204685
:10566000FFF746FEAA0303D501212046FFF740FEBF
:105670006B0303D502212046FFF73AFE2F0303D523
:1056800003212046FFF734FEE80203D5042120461B
:10569000FFF72EFEA90203D505212046FFF728FEBD
:1056A0006A0203D506212046FFF722FE2B0203D50E
:1056B00007212046FFF71CFEEF0103D508212046F5
:1056C000FFF716FE700340F1A780E90703D500211C
:1056D0002046FFF79FFEAA0703D501212046FFF7CA
:1056E00099FE6B0703D502212046FFF793FE2F0793
:1056F00003D503212046FFF78DFEEE0603D50421D6
:105700002046FFF787FEA80603D505212046FFF7B0
:1057100081FE690603D506212046FFF77BFE2A0697
:1057200003D507212046FFF775FEEB0574D520460B
:105730000821BDE8F84FFFF76DBED4F890904FF008
:10574000000B4FF0010AD4F894305FFA8BF79B6896
:105750009F423FF638AF09EB4713D3F8002902F414
:105760004022B2F5802F20D1D3F80029002A1CDA7C
:10577000D3F8002942F09042C3F80029D3F8002959
:10578000002AFBDB3946D4F89000FFF787FB22891B
:105790000AFA07F322EA0303238104EB8703DB6899
:1057A0009B6813B13946204698470BF1010BCAE7B5
:1057B000910701D1D0F80080072A02F101029CBFB5
:1057C00003F8018B4FEA18283FE704EB830300F549
:1057D0008050DA68D2F818C0DCF80820DCE9001C38
:1057E000A1EB0C0C00218F4208D1DB689B699A6801
:1057F0003A449A605A683A445A6029E711F0030F14
:1058000001D1D0F800808C4501F1010184BF02F87C
:10581000018B4FEA1828E6E7BDE8F88F08B5034882
:10582000FFF774FEBDE8084000F06CBCB8480020EB
:1058300008B50348FFF76AFEBDE8084000F062BC07
:1058400054490020D0F8903003EB4111D1F8003BCF
:1058500043F40013C1F8003B70470000D0F89030CB
:1058600003EB4111D1F8003943F40013C1F80039BA
:1058700070470000D0F8903003EB4111D1F8003BA5
:1058800023F40013C1F8003B70470000D0F89030BB
:1058900003EB4111D1F8003923F40013C1F80039AA
:1058A00070470000090100F16043012203F56143E4
:1058B000C9B283F8001300F01F039A4043099B000C
:1058C00003F1604303F56143C3F880211A60704718
:1058D00030B50433039C0172002104FB0325C16031
:1058E000C0E90653049B0363059BC0E90000C0E9BF
:1058F0000422C0E90842C0E90A11436330BD000038
:105900000022416AC260C0E90411C0E90A226FF0B6
:105910000101FEF767BB0000D0E90432934201D1D8
:10592000C2680AB9181D70470020704703691960E2
:105930000021C2680132C260C26913448269934285
:10594000036124BF436A0361FEF740BB38B50446D8
:105950000D46E3683BB162690020131D1268A36223
:105960001344E36207E0237A33B929462046FEF761
:105970001DFB0028EDDA38BD6FF00100FBE70000E9
:10598000C368C269013BC36043691344826993429F
:10599000436124BF436A436100238362036B03B105
:1059A0001847704770B53023044683F31188866A20
:1059B0003EB9FFF7CBFF054618B186F3118828469C
:1059C00070BDA36AE26A13F8015B9342A36202D33B
:1059D0002046FFF7D5FF002383F31188EFE700008F
:1059E0002DE9F84F04460E46174698464FF0300909
:1059F00089F311880025AA46D4F828B0BBF1000F1E
:105A000009D141462046FFF7A1FF20B18BF3118851
:105A10002846BDE8F88FD4E90A12A7EB050B521A05
:105A2000934528BF9346BBF1400F1BD9334601F184
:105A3000400251F8040B914243F8040BF9D1A36AD8
:105A4000403640354033A362D4E90A239A4202D358
:105A50002046FFF795FF8AF31188BD42D8D289F31B
:105A60001188C9E730465A46FBF77EFDA36A5E44BB
:105A70005D445B44A362E7E710B5029C0433017206
:105A800003FB0421C460C0E906130023C0E90A3304
:105A9000039B0363049BC0E90000C0E90422C0E942
:105AA0000842436310BD0000026A6FF00101C2604A
:105AB000426AC0E904220022C0E90A22FEF792BA33
:105AC000D0E904239A4201D1C26822B9184650F89D
:105AD000043B0B60704700231846FAE7C3680021B7
:105AE000C2690133C36043691344826993424361CD
:105AF00024BF436A4361FEF769BA000038B5044623
:105B00000D46E3683BB1236900201A1DA262E269D9
:105B10001344E36207E0237A33B929462046FEF7AF
:105B200045FA0028EDDA38BD6FF00100FBE7000010
:105B300003691960C268013AC260C269134482698C
:105B40009342036124BF436A036100238362036BB2
:105B500003B118477047000070B530230D46044666
:105B6000114683F31188866A2EB9FFF7C7FF10B17B
:105B700086F3118870BDA36A1D70A36AE26A0133BF
:105B80009342A36204D3E16920460439FFF7D0FFB2
:105B9000002080F31188EDE72DE9F84F04460D460B
:105BA000904699464FF0300A8AF311880026B34692
:105BB000A76A4FB949462046FFF7A0FF20B187F3F7
:105BC00011883046BDE8F88FD4E90A073A1AA8EBE5
:105BD0000607974228BF1746402F1BD905F14003FF
:105BE00055F8042B9D4240F8042BF9D1A36A4036A6
:105BF0004033A362D4E90A239A4204D3E1692046E0
:105C00000439FFF795FF8BF311884645D9D28AF303
:105C10001188CDE729463A46FBF7A6FCA36A3D4426
:105C20003E443B44A362E5E7D0E904239A4217D1FE
:105C3000C3689BB1836A8BB1043B9B1A0ED013607F
:105C4000C368013BC360C3691A4483699A42026115
:105C500024BF436A0361002383620123184670470F
:105C60000023FBE700F078BA014B586A704700BF89
:105C7000000C0040034B002258631A610222DA60D4
:105C8000704700BF000C0040014B0022DA607047F3
:105C9000000C0040014B5863704700BF000C0040EF
:105CA000024B034A1A60034A5A607047084A0020B0
:105CB000B04A002000000220074B494210B55C6842
:105CC000201A08401968821A8A4203D3A24201D8D6
:105CD0005A6010BD0020FCE7084A002008B53023B8
:105CE00083F31188FFF7E8FF002383F3118808BDD1
:105CF00004480121044B03600023C0E901330C3048
:105D0000FEF766B8104A0020DD5C0008CB1D083A9B
:105D100023F00703591A521A012110B4D2080024A3
:105D2000C0E9004384600C301C605A605DF8044B8D
:105D3000FEF74EB82DE9F84F364ECD1D0F46002820
:105D400018BF0646082A4FEAD50538BF082206F1D3
:105D50000C08341D91464046FEF756F809F107013C
:105D6000C9F1000E224624686CB94046FEF756F889
:105D70003368CBB308224946E8009847044698B3F5
:105D800040E9026730E004EB010CD4F804A00CEA0F
:105D90000E0C0AF10100ACF1080304EBC0009842BC
:105DA000E0D9A0EB0C0CB5EBEC0F4FEAEC0BD9D81B
:105DB0009C421CD204F10802AB45A3EB02024FEA5D
:105DC000E202626009D9691CED43206803EBC1025D
:105DD0005D44556043F8310022601C465F604046D8
:105DE00044F8086BFEF71AF82046BDE8F88FAA457C
:105DF000216802D111602346EFE7013504EBC503AA
:105E000044F8351003F10801401AC01058601360BF
:105E1000F1E700BF104A0020F8B550F8043C0446F2
:105E200050F8085CA0F1080607332F1D0C35DB087D
:105E300040F8043C2846FDF7E7FF3B469F421A68BE
:105E400001D0B34228D20AB1964225D244F8082C98
:105E500054F8042C1E60013254F8081C06EBC200F2
:105E6000814206D14868024444F8042C0A6844F888
:105E7000082C5868411C03EBC1018E4207D154F82D
:105E8000042C013202445A6054F8082C1A60284647
:105E9000BDE8F840FDF7C2BF1346CFE7FEE70000BC
:105EA00070B51B4B0025044686B058600E468562CF
:105EB000016300F0FFF804F11003A560E562C4E996
:105EC00004334FF0FF33C4E90044C4E90635FFF75B
:105ED000CBFE2B46024604F134012046C4E90823D8
:105EE00080230C4A2565FDF7FFFF01230A4AE06085
:105EF00000920375684672680192B268CDE9022388
:105F0000064BCDE90435FEF717F806B070BD00BFAB
:105F1000F82B0020606D0008656D00089D5E00088C
:105F2000024AD36A1843D062704700BF902900200C
:105F30004B6843608B688360CB68C3600B694361C7
:105F40004B6903628B6943620B6803607047000012
:105F500008B5354B40F2FF70D3F8E0100143C3F8A9
:105F6000E010D3F8082102433048C3F80821304A32
:105F7000D3F808311146FFF7DBFF00F5806002F12E
:105F80001C01FFF7D5FF00F5806002F13801FFF733
:105F9000CFFF00F5806002F15401FFF7C9FF00F563
:105FA000806002F17001FFF7C3FF00F5806002F12D
:105FB0008C01FFF7BDFF00F5806002F1A801FFF73B
:105FC000B7FF00F5806002F1C401FFF7B1FF00F5F3
:105FD000806002F1E001FFF7ABFF00F5806002F1A5
:105FE000FC01FFF7A5FF02F58C7100F58060FFF75B
:105FF0009FFF00F07DF90F4BD3F8902242F0010291
:10600000C3F89022D3F8942242F00102C3F89422FC
:106010000522C3F898204FF06052C3F89C20064A2E
:10602000C3F8A02008BD00BF004402580000025879
:106030006C6D000800ED00E01F00080308B500F0DB
:1060400045FBFDF701FF104BD3F8DC2042F0400286
:10605000C3F8DC20D3F8042122F04002C3F8042165
:10606000D3F80431094B1A6842F008021A601A6822
:1060700042F004021A60FEF753FDFEF7BDFBBDE8D7
:106080000840FEF79BB900BF0044025800180248C0
:1060900070470000EFF30983054968334A6B22F02B
:1060A00001024A6383F30988002383F31188704750
:1060B00000EF00E0302080F3118862B60D4B0E4AED
:1060C000D96821F4E0610904090C0A430B49DA603C
:1060D000D3F8FC2042F08072C3F8FC20084AC2F8D2
:1060E000B01F116841F0010111602022DA7783F8B6
:1060F0002200704700ED00E00003FA0555CEACC564
:10610000001000E0302310B583F311880E4B5B685C
:1061100013F4006314D0F1EE103AEFF309844FF05A
:106120008073683CE361094BDB6B236684F3098869
:10613000FDF722FE10B1064BA36110BD054BFBE736
:1061400083F31188F9E700BF00ED00E000EF00E005
:106150004307000846070008114BD3F8E82042F037
:106160000802C3F8E820D3F8102142F00802C3F86F
:1061700010210C4AD3F81031D36B43F00803D363DA
:10618000C722094B9A624FF0FF32DA6200229A610D
:106190005A63DA605A6001225A611A60704700BF80
:1061A000004402580010005C000C0040094A08B589
:1061B0001169D3680B40D9B29B076FEA01011161E5
:1061C00007D5302383F31188FDF768FE002383F39E
:1061D000118808BD000C0040064BD3F8DC200243B8
:1061E000C3F8DC20D3F804211043C3F80401D3F82A
:1061F000043170470044025808B53C4B4FF0FF3162
:10620000D3F8802062F00042C3F88020D3F88020C9
:1062100002F00042C3F88020D3F88020D3F8842015
:10622000C3F88410D3F884200022C3F88420D3F864
:106230008400D86F40F0FF4040F4FF0040F4DF409E
:1062400040F07F00D867D86F20F0FF4020F4FF00B7
:1062500020F4DF4020F07F00D867D86FD3F88800A3
:106260006FEA40506FEA5050C3F88800D3F88800B6
:10627000C0F30A00C3F88800D3F88800D3F8900070
:10628000C3F89010D3F89000C3F89020D3F8900092
:10629000D3F89400C3F89410D3F89400C3F8942072
:1062A000D3F89400D3F89800C3F89810D3F8980066
:1062B000C3F89820D3F89800D3F88C00C3F88C105A
:1062C000D3F88C00C3F88C20D3F88C00D3F89C0052
:1062D000C3F89C10D3F89C10C3F89C20D3F89C30D2
:1062E000FEF744FDBDE8084000F0C0B90044025884
:1062F00008B50122534BC3F80821534BD3F8F420BF
:1063000042F00202C3F8F420D3F81C2142F002024A
:10631000C3F81C210222D3F81C314C4BDA605A68B6
:106320009104FCD54A4A1A6001229A60494ADA600F
:1063300000221A614FF440429A61444B9A699204D8
:10634000FCD51A6842F480721A603F4B1A6F12F43F
:10635000407F04D04FF480321A6700221A671A680F
:1063600042F001021A60384B1A685007FCD500222F
:106370001A611A6912F03802FBD1012119604FF03D
:10638000804159605A67344ADA62344A1A611A689D
:1063900042F480321A602C4B1A689103FCD51A68BB
:1063A00042F480521A601A689204FCD52C4A2D4996
:1063B0009A6200225A63196301F57C01DA6301F2E3
:1063C000E71199635A64284A1A64284ADA621A68FB
:1063D00042F0A8521A601C4B1A6802F02852B2F11F
:1063E000285FF9D148229A614FF48862DA6140222D
:1063F0001A624FF00052DA641D4A1A651D4A5A6546
:106400001D4A9A6532231D4A1360136803F00F0377
:10641000022BFAD10C4A136943F003031361136989
:1064200003F03803182BFAD14FF00050FFF7D4FED9
:106430004FF08040FFF7D0FE4FF00040BDE808402D
:10644000FFF7CABE008000510044025800480258BD
:1064500000C000F0020000010000FF010088900869
:106460002220400063020901470E0508DD0BBF0131
:10647000000001100910E00000010110002000528E
:106480004FF0B04208B5D2F8883003F00103C2F8EB
:10649000883023B1044A13680BB150689847BDE8AF
:1064A0000840FFF72FBE00BF284A00204FF0B0423F
:1064B00008B5D2F8883003F00203C2F8883023B15F
:1064C000044A93680BB1D0689847BDE80840FFF7CD
:1064D00019BE00BF284A00204FF0B04208B5D2F8DC
:1064E000883003F00403C2F8883023B1044A1369EA
:1064F0000BB150699847BDE80840FFF703BE00BFE5
:10650000284A00204FF0B04208B5D2F8883003F096
:106510000803C2F8883023B1044A93690BB1D069EB
:106520009847BDE80840FFF7EDBD00BF284A0020AE
:106530004FF0B04208B5D2F8883003F01003C2F82B
:10654000883023B1044A136A0BB1506A9847BDE8FA
:106550000840FFF7D7BD00BF284A00204FF0B043E6
:1065600010B5D3F8884004F47872C3F88820A306E5
:1065700004D5124A936A0BB1D06A9847600604D5D5
:106580000E4A136B0BB1506B9847210604D50B4A8A
:10659000936B0BB1D06B9847E20504D5074A136C97
:1065A0000BB1506C9847A30504D5044A936C0BB10A
:1065B000D06C9847BDE81040FFF7A4BD284A0020E2
:1065C0004FF0B04310B5D3F8884004F47C42C3F8D0
:1065D0008820620504D5164A136D0BB1506D98479B
:1065E000230504D5124A936D0BB1D06D9847E00492
:1065F00004D50F4A136E0BB1506E9847A10404D511
:106600000B4A936E0BB1D06E9847620404D5084ACA
:10661000136F0BB1506F9847230404D5044A936F4E
:106620000BB1D06F9847BDE81040FFF76BBD00BFBE
:10663000284A002008B50348FCF75AFBBDE808408B
:10664000FFF760BD0425002008B50348FCF702FCF5
:10665000BDE80840FFF756BD2425002008B5FFF728
:10666000A5FDBDE80840FFF74DBD0000062108B5B7
:106670000846FFF717F906210720FFF713F906214F
:106680000820FFF70FF906210920FFF70BF9062173
:106690000A20FFF707F906211720FFF703F9062163
:1066A0002820FFF7FFF809217A20FFF7FBF80A21DD
:1066B0005C20FFF7F7F807213220FFF7F3F80C21F1
:1066C0005220BDE80840FFF7EDB8000008B5FFF71D
:1066D00093FD00F00FF8FCF7D5FDFCF7ADFFFCF7DC
:1066E0007FFEFDF743FAFFF7D3FCBDE80840FFF754
:1066F000B9BA00000023054A19460133102BC2E93C
:10670000001102F10802F8D1704700BF284A0020AA
:106710000B460146184600F027B80000FEF7A4B863
:10672000FFF7FCBF012838BF012010B50446204602
:10673000FEF75AF830B900F007F808B900F00CF885
:106740008047F4E710BD0000024B1868BFF35B8F71
:10675000704700BFA84A002008B5062000F04AF89C
:106760000120FDF779FD000010B5054C13462CB152
:106770000A4601460220AFF3008010BD2046FCE728
:106780000000000010B501390244904201D1002000
:1067900005E0037811F8014FA34201D0181B10BD8A
:1067A0000130F2E71F2938B504460D4604D91623F7
:1067B00003604FF0FF3038BD426C12B152F8213007
:1067C0004BB9204600F030F82A4601462046BDE885
:1067D000384000F017B8012B0AD0591C03D11623FA
:1067E00003600120E7E7002442F825402846984747
:1067F0000020E0E7024B01461868FFF7D3BF00BF57
:106800006422002038B5074D00230446084611468F
:106810002B60FDF725FD431C02D12B6803B12360DB
:1068200038BD00BFAC4A0020FDF714BD034611F887
:10683000012B03F8012B002AF9D17047000000005A
:106840000100000000010001000000000000000045
:106850000000000052657175657374656420746F83
:10686000206572617365206D6F7265207468616E5A
:106870002077652063616E0A00457261736520436D
:106880006F6D6D616E642052656365697665640A3B
:106890000050435420444F4E453A2025640A0000DE
:1068A00053544D333248373F3F3F0053544D3332FA
:1068B000483733782F3732780053544D33324837C6
:1068C00034332F3735332F373530000001105A005D
:1068D000031059000120580003205600534644502D
:1068E000000000004A454445433A204661696C6512
:1068F0006420746F2064657465637420666C6173D2
:1069000068206465766963653A2025730A004A4504
:106910004445433A204661696C656420746F206386
:106920006F6E66696720666C61736820646576695E
:1069300063653A2025730A004A454445433A20449A
:106940006574656374656420466C61736820446592
:10695000766963653A2025730A0045787420466C91
:10696000617368204E6F7420466F756E642100005D
:106970006D74323571007732357100773235712D93
:10698000647472007069000820BA00000000000002
:1069900076690008EF400000000000007B690008F5
:1069A000EF70000000000000000000000000000088
:1069B000211E0008892000083D1700084117000823
:1069C000E9170008F11F00084517000849170008DB
:1069D000E91E0008B9170008491F00082D1C00080F
:1069E000511700084D17000821210008B1170008B1
:1069F0000000000000000000000000000000000097
:106A00001922000861250008612500081D220008E0
:106A100021220008252200082922000861250008FB
:106A20006125000861250008412200084522000870
:106A30005D22000865220008712200087522000806
:106A40007922000804250020010000000000000059
:106A500000000000B1230008C92300081922000823
:106A600085220008FD230008B922000895240008AB
:106A7000C5240008292200089D2200088922000858
:106A80009922000841220008452200085D220008E2
:106A9000652200087122000875220008792200088A
:106AA000A1220008000000000000000031230008BF
:106AB0007D22000881220008000000000000000084
:106AC0002926000831260008152600081D26000882
:106AD0004126000845260008286E756C6C290000C8
:106AE00000000000C52A00089D2A00084D2A000861
:106AF000692A0008852A00084D444D4120666169D5
:106B00006C75726500000000009600000000000037
:106B10000000000000000000000000000000000075
:106B20000000000045320008313200086D320008D4
:106B30005932000865320008513200083D32000821
:106B40002932000879320008000000005D33000897
:106B50004933000885330008713300087D3300088D
:106B600069330008553300084133000891330008A9
:106B70000000000001000000000000006330000081
:106B80007C6B0008E8290020F82B00204172647516
:106B900050696C6F740025424F415244252D424C80
:106BA000002553455249414C2500000002000000D9
:106BB000000000007D350008ED3500084000400071
:106BC000A8440020B844002002000000000000009B
:106BD000030000000000000035360008000000003F
:106BE00010000000C8440020000000000100000068
:106BF00000000000B84800200101020059430008CD
:106C00006942000805430008E9420008430000000B
:106C1000146C000809024300020100C0320904009C
:106C200000010202010005240010010524010001F9
:106C3000042402020524060001070582030800FF60
:106C400009040100020A00000007050102400000DB
:106C5000070581024000000012000000606C00087F
:106C60001201100102000040091241570002010206
:106C7000030100000403090425424F41524425004A
:106C8000594A5541565F413653450030313233340D
:106C9000353637383941424344454600000000202C
:106CA00000000200020000000000003000000400AC
:106CB00000000000000000240000080004000000A4
:106CC0000004000000FC000002000000000004308E
:106CD00000800000000000000000003800000100FB
:106CE000010000004000005280000052C00000522D
:106CF000000100524001005280010052C0010052C8
:106D0000000200524002005280020052C0020052B3
:106D1000000300524003005280030052C00300529F
:106D2000000400520000000091370008493A0008B2
:106D3000F53A000840004000F0490020F0490020EA
:106D400001000000004A0020800000004001000017
:106D50000800000000010000001000000800000012
:106D60006D61696E0069646C650000000100802A35
:106D700000000000AAAAAAAA01000024FFFF000048
:106D80000000000000A00A00202000000000000019
:106D9000BABAAAAA00000000FFFF00000009000A1A
:106DA000000000000000004000000000AAAAAAAAFB
:106DB00000000040FFFF0000000000000000000095
:106DC0000000900A00040000AAAAEAAF0000000038
:106DD000FFFF000000000000009099006085164051
:106DE00000800000BAAAAAAA40451500FFFF0000D3
:106DF0000009007007000000000000000000000013
:106E0000AAAAAAAA00000000FFFF000000000000DC
:106E1000000000000100000001000000AAAAAAAAC8
:106E200000000000FFFF0000000000000000000064
:106E30000000000000000000AAAAAAAA00000000AA
:106E4000FFFF000000000000000000000000000044
:106E500000000000AAAAAAAA00000000FFFF00008C
:106E60000000000000000000000000000000000022
:106E7000AAAAAAAA00000000FFFF0000000000006C
:106E8000000000000000000000000000AAAAAAAA5A
:106E900000000000FFFF00000000000000000000F4
:106EA0008094FF7F010000006704000000000000E4
:106EB000000000000000E900FF000000002C00209E
:106EC0002425002000000000A068000883040000C2
:106ED000AB68000850040000B96800080096000084
:106EE00000000800960000000008000004000000F8
:106EF000746C0008000000000000000000000000AA
:106F000000000000000000000000000068220020D7
:106F10000000000000000000000000000000000071
:106F20000000000000000000000000000000000061
:106F30000000000000000000000000000000000051
:106F40000000000000000000000000000000000041
:106F50000000000000000000000000000000000031
:106F60000000000000000000000000000000000021
:00000001FF
